S01500006376615F6173775F6D303131382E7372656395
S214010000F05F002069A901002B4201007B4201003C
S21401001000000000000000000000000000000000DA
S214010020000000000000000000000000674301001F
S21401003000000000000000004F45010037A301004A
S214010040C0AC0100C0AC0100C0AC0100C0AC0100F6
S214010050C0AC0100C0AC0100C0AC0100C0AC0100E6
S214010060C0AC010051640100C0AC0100C0AC01008D
S214010070C0AC0100C0AC0100C0AC0100C0AC0100C6
S214010080C0AC0100C0AC0100C0AC0100C0AC0100B6
S214010090C0AC0100C0AC0100C0AC0100C0AC0100A6
S2140100A0C0AC0100C0AC0100C0AC0100C0AC010096
S2140100B0C0AC0100C0AC0100C0AC0100C0AC010086
S2140100C0DDCCBBAA31343A30393A34340000000072
S2140100D046656220203520323032350000000000AF
S2140100E05357303130315F323032353032303400B0
S2140100F000000000000000000000000000000000FA
S21401010000B583680122DB681340DBB2002B0AD0FE
S21401011083681B6A9B081A40D2B2002A03D0C069C2
S2140101200860012000E0002000BD70B500231C001F
S2140101308568EE68012296430122E4B214403443F6
S214010140EC600978002943D0C169224CA14201D153
S2140101501D0012E0C169BA4CA14201D215000CE0A3
S214010160C169B84CA14201D2022506E0C169B64C6C
S214010170A14201D2032500E004252900C9B20429C1
S21401018001D1002025E08168CC680C26B443EDB28D
S214010190AE000C2535402543CD608168CC6810251E
S2140101A0AC43DBB21B0110252B402343CB6011006F
S2140101B08368DC680125AC43C9B211402143D9608C
S2140101C08168096A8B0811001940C9B20029F7D065
S2140101D0012070BD00093D0000B58268126A53080F
S2140101E01A00D207D20FD2B2002A03D08069086063
S2140101F0012000E0002000BD7CB504000D000020B9
S214010200A16801264A6931001140C9B200295BD0B4
S214010210A1680A6A31001140C9B2002954D0A16808
S21401022089690A0931001140C9B2002902D00129A1
S21401023005D009E069462000FFF762FF04E0694641
S2140102402000FFF7C9FFFFE7C0B2002801D1002058
S2140102503BE03100A0684069000A8007800FC0B209
S214010260002805D0022807D004D3032806D007E0CB
S214010270310005E0022103E0042101E00821FFE747
S214010280A0684069400843065B0EDBB2002B01D133
S2140102908023FFE7A0684069C00A4207520FD2B226
S2140102A0002A01D10822FFE7A0684069800A3400CD
S2140102B00440E4B2641C009858436043514349002B
S2140102C002F0DFFC28603000C0B276BDF1B5002434
S2140102D02000009A9268556901239D430123C0B20C
S2140102E018402843506118004A78002A02D0012A93
S2140102F00DD019E02600009A9568AA691027BA431E
S214010300F6B2360110273E401643AE610DE01E00E0
S214010310009A9568AA691027BA43F6B236011027E3
S2140103203E401643AE6100E020000200D2B2002A31
S21401033001D1002081E0CA68012A01D126000FE020
S214010340CA68022A01D11E000AE0CA68042A01D13D
S214010350022605E0CA68082A01D1032600E0FF2626
S2140103603200D2B2FF2A01D1002066E0009A9268DC
S2140103705769BD4D3D40F6B23702C026B6003E4035
S2140103802E4356614A88002A18D04A88812A15DAEF
S2140103904A88802A01D1220000E04A88009DAD6883
S2140103A06E69FE27BE43D2B25700FE223A40324360
S2140103B06A610A69002A03D100203EE000203CE081
S2140103C00A69092AF8D20A69082A00D00C69009A33
S2140103D092685669A54D3540E4B2E602E024A401D0
S2140103E034402C4354618A68012A02D08A68022A62
S2140103F024D18D686D1E009A926856699C4C3440D3
S214010400EDB2AD028026F6003540254355610978E8
S214010410002911D01900009A926854690125AC434D
S214010420C9B2194021435161009989680A6A1900C5
S2140104301140C9B20029F7D0C0B2F2BD0020FCE7D6
S21401044001127A0001366E01015A6202F8B5040003
S2140104500E0000270020009060690125C06901098F
S21401046028000840C0B2002817D069462000FFF7D0
S21401047047FE07003800C0B200280ED06069C06988
S214010480000A4007400F85402900412904D2009800
S21401049002F0F7FB306000E000273800C0B2F2BD82
S2140104A0FCB500226B461A7016004569EF691023E9
S2140104B0DB431F401024F6B2360126403E43EE6170
S2140104C08D88012D01D115001EE08D88022D01D1E8
S2140104D0012519E08D88042D01D1022514E08D88AF
S2140104E0082D01D103250FE08D88102D01D104259B
S2140104F00AE08D88202D01D1052505E08D88402D47
S21401050001D1062500E007252E00F6B2072E14D0ED
S2140105106E4635704569EF699A4E3E400196019FD9
S214010520BC466E4636783702E026F6003E40674601
S2140105303E43EE6101256E4635700978002901D0EB
S2140105400122FFE74069C1690B40D2B211010C409C
S2140105501C43C46168460078F6BDF8B504000E0079
S21401056000270020009060690125806901092800A4
S2140105700840C0B2002817D069462000FFF7C0FD2A
S21401058007003800C0B200280ED060698069000AF2
S2140105904007400F85402900412904D2009802F007
S2140105A070FB306000E000273800C0B2F2BDFCB539
S2140105B000226B461A7016004569AF691023DB43AB
S2140105C01F401024F6B2360126403E43AE618D88A8
S2140105D0012D01D115001EE08D88022D01D10125C6
S2140105E019E08D88042D01D1022514E08D88082D8F
S2140105F001D103250FE08D88102D01D104250AE0D5
S2140106008D88202D01D1052505E08D88402D01D14D
S214010610062500E007252E00F6B2072E14D06E46FA
S21401062035704569AF69574E3E400196019FBC46FD
S2140106306E4636783702E026F6003E4067463E4371
S214010640AE6101256E4635700978002901D0012278
S214010650FFE7406981690B40D2B211010C401C438F
S214010660846168460078F6BDFFFCFFFFFFC7FFFF09
S214010670FFFBFFFFF8B504000E00002700200090E6
S214010680606901254069010928000840C0B20028B8
S21401069017D069462000FFF79FFD07003800C0B25B
S2140106A000280ED060694069000A4007400F854067
S2140106B02900412904D2009802F0E3FA306000E0F4
S2140106C000273800C0B2F2BDFCB500226B461A7096
S2140106D0160045696F691023DB431F401024F6B2EC
S2140106E0360126403E436E618D88012D01D11500ED
S2140106F01EE08D88022D01D1012519E08D88042D7B
S21401070001D1022514E08D88082D01D103250FE0C3
S2140107108D88102D01D104250AE08D88202D01D168
S214010720052505E08D88402D01D1062500E0072529
S2140107302E00F6B2072E14D06E46357045696F69E5
S214010740104E3E400196019FBC466E4636783702F3
S214010750E026F6003E4067463E436E6101256E4642
S21401076035700978002901D00122FFE74069416907
S2140107700B40D2B211010C401C434461684600781C
S214010780F6BD0000FFF8FFFFF8B504000E000027D5
S21401079000200090606901250069010928000840D1
S2140107A0C0B2002817D069462000FFF715FD0700E4
S2140107B03800C0B200280ED060690069000A400700
S2140107C0400F85402900412904D2009802F059FAC9
S2140107D0306000E000273800C0B2F2BDFCB5002250
S2140107E06B461A70160045692F691023DB431F40BC
S2140107F01024F6B2360126403E432E618D88012D27
S21401080001D115001EE08D88022D01D1012519E0C8
S2140108108D88042D01D1022514E08D88082D01D183
S21401082003250FE08D88102D01D104250AE08D885F
S214010830202D01D1052505E08D88402D01D1062505
S21401084000E007252E00F6B2072E14D06E4635704E
S21401085045692F69974E3E400196019FBC466E46FC
S21401086036783702E026F6003E4067463E432E6164
S21401087001256E4635700978002901D00122FFE76F
S214010880406901690B40D2B211010C401C4304615E
S21401089068460078F6BDF8B504000E000027002073
S2140108A0009060690125406A010928000840C0B22D
S2140108B0002817D069462000FFF79EFC0700380085
S2140108C0C0B200280ED06069406A000A4007400F97
S2140108D085402900412904D2009802F0D2F93060FF
S2140108E000E000273800C0B2F2BDFCB500226B461E
S2140108F01A70160045696F6A1023DB431F401024E7
S214010900F6B2360126403E436E628D88012D01D136
S21401091015001EE08D88022D01D1012519E08D8874
S214010920042D01D1022514E08D88082D01D103255F
S2140109300FE08D88102D01D104250AE08D88202D29
S21401094001D1052505E08D88402D01D1062500E061
S21401095007252E00F6B2072E14D06E46357045696F
S2140109606F6A544E3E400196019FBC466E463678ED
S2140109703702E026F6003E4067463E436E6201259A
S2140109806E4635700978002901D00122FFE74069DB
S214010990416A0B40D2B211010C401C4344626846C6
S2140109A00078F6BDF8B504000E0000270020009080
S2140109B060690125006A010928000840C0B20028C4
S2140109C017D069462000FFF717FC07003800C0B2B1
S2140109D000280ED06069006A000A4007400F854073
S2140109E02900412904D2009802F04BF9306000E05A
S2140109F000273800C0B2F2BDFCB500226B461A7063
S214010A00160045692F6A1023DB431F401024F6B2F7
S214010A10360126403E432E628D88012D01D11500F8
S214010A201EE08D88022D01D1012519E08D88042D47
S214010A3001D1022514E08D88082D01D103250FE090
S214010A408D88102D01D104250AE08D88202D01D135
S214010A50052505E08D88402D01D1062500E00725F6
S214010A602E00F6B2072E14D06E46357045692F6AF1
S214010A70104E3E400196019FBC466E4636783702C0
S214010A80E026F6003E4067463E432E6201256E464E
S214010A9035700978002901D00122FFE74069016A13
S214010AA00B40D2B211010C401C4304626846007828
S214010AB0F6BD0000FFF8FFFF80B50A00002143697C
S214010AC01B681B0E9B079B0FDBB2002B05D0022B6E
S214010AD00DD007D3032B0FD013E01100FFF77CFBDB
S214010AE001000EE01100FFF70BFB010009E0110009
S214010AF0FFF782FB010004E01100FFF76DFB010028
S214010B00FFE70800C0B202BD30B54A78012A01D11C
S214010B1000210AE04A78002A01D1012105E049783E
S214010B20022901D1022100E0FF210A00D2B2FF2AE8
S214010B3001D1002016E00A0043691C688B4D254050
S214010B40D2B21404C022920222402A431A60426999
S214010B501268120E9207920F0B00D2B2DBB29A42C3
S214010B60F5D1012030BD7CB504000D00002069469A
S214010B702000FFF7A1FF06003000C0B2002801D117
S214010B8000200BE0E06800680107090F0098C9B271
S214010B90491C02F076F828603000C0B276BD00B578
S214010BA08A88002A0FD08A88112A0CDA8988491E79
S214010BB0C06802680F239A43C9B20907090F114397
S214010BC00160012000E0002000BD7CB504000D009E
S214010BD0002069462000FFF7C6FF06003000C0B2BD
S214010BE0002801D100200CE060690068000A0107B6
S214010BF0090F0098C9B2491C02F043F8286030007A
S214010C00C0B276BD00B58A88002A11D08A88112A1A
S214010C100EDA8988491E40690268554B1340C9B2ED
S214010C200A02F0210901114019430160012000E088
S214010C30002000BDF8B504000D000026370020692D
S214010C40C8214058000C8007800FC0B2002805D08C
S214010C5002280FD008D3032812D017E069462000D7
S214010C60FFF7BAFA070011E069462000FFF748FAD5
S214010C7007000BE069462000FFF7BEFA070005E013
S214010C8069462000FFF7A8FA0700FFE73800C0B260
S214010C90002801D1002019E02069C8214058010927
S214010CA00800C007C00FC0B200280CD02069C821B8
S214010CB04058000A0107090F0098C9B2491C01F003
S214010CC0E0FF286000E037003800C0B2F2BD30B562
S214010CD04A78012A01D100220AE04A78002A01D185
S214010CE0012205E04A78022A01D1022200E0FF2211
S214010CF01300DBB2FF2B01D1002036E08B88002BDE
S214010D0032D08B88112B2FDA0369C8241C59174D52
S214010D102540D2B21404C022920222402A43C8249B
S214010D201A518B885B1E0269C8241459104D254040
S214010D30DBB21C02F0231B0123402B43C8241351B2
S214010D400978002901D0012100E000210069C822AC
S214010D50825810239A43C9B209011023194011433E
S214010D60C8228150012000E0002030BDFFFFFCFFBB
S214010D70FFF0FFFFF8B504000D0060694068010947
S214010D800800C007C00FC0B2002801D100209BE0B8
S214010D90002007000090606907264068000C30407C
S214010DA0C0B2002843D160694068C00C3040C0B270
S214010DB000280BD0022815D00ED304281ED017D336
S214010DC0062827D020D307282AD02FE069462000FE
S214010DD0FFF730FF070066E069462000FFF790F94D
S214010DE0070060E069462000FFF7F6F907005AE0C1
S214010DF069462000FFF700FA070054E06946200024
S214010E00FFF7B1FE07004EE069462000FFF7DDFE62
S214010E10070048E069462000FFF718FB070042E09C
S214010E2069462000FFF726FC07003CE03BE06069CE
S214010E304068000C3040C0B201280AD033D30328E2
S214010E4013D00CD305281CD015D3072825D01ED3C4
S214010E5029E069462000FFF71EFD070023E06946EA
S214010E60200000F0EFF907001DE06946200000F0C1
S214010E70C5F9070017E06946200000F09BF9070056
S214010E8011E06946200000F0ABFC07000BE0694664
S214010E902000FFF7A1F9070005E069462000FFF7EB
S214010EA09BF90700FFE73800C0B201280AD1606944
S214010EB04068000A064031000098C9B2491C01F09A
S214010EC0E0FE28603800C0B2F2BDF2B50123190079
S214010ED00024260045696A681027BA43F6B236012F
S214010EE010273E4016436E60009A5278002A39D089
S214010EF0012A50D0022A67D0032A00D1AFE0052A82
S214010F0000D1C5E0072A00D1DBE00A2A75D00B2AFA
S214010F1000D18BE00C2A0CD00F2A00D1F8E0102A61
S214010F2000D1E8E0112A00D1D8E01A2A00D1FCE06D
S214010F3008E12600426957689A4D3D40F6B23704EB
S214010F40E026F6023E402E43566026004269576868
S214010F50954D3D40F6B2F704E026B6033E402E43DB
S214010F605660F0E02600426957688E4D3D40F6B265
S214010F703704E026F6023E402E4356601E004269C4
S214010F805768894D3D40F6B2F704E026B6033E4069
S214010F902E435660D7E0260042695768814D3D4092
S214010FA0F6B23704E026F6023E402E43566002268D
S214010FB0426957687C4D3D40F6B2F704E026B60319
S214010FC03E402E435660BEE0260042695768754D86
S214010FD03D40F6B23704E026F6023E402E43566008
S214010FE0032642695768704D3D40F6B2F704E02685
S214010FF0B6033E402E435660A5E026004269576878
S214011000684D3D40F6B23704E026F6023E402E43D8
S2140110105660042642695768634D3D40F6B2F704B0
S214011020E026B6033E402E4356608CE02600426919
S21401103057685C4D3D40F6B23704E026F6023E4066
S2140110402E435660052642695768574D3D40F6B215
S214011050F704E026B6033E402E43566073E02600B2
S214011060426957684F4D3D40F6B23704E026F60216
S2140110703E402E4356600626426957684A4D3D401B
S214011080F6B2F704E026B6033E402E4356605AE019
S214011090260042695768434D3D40F6B23704E026C4
S2140110A0F6023E402E4356600726426957683E4D7B
S2140110B03D40F6B2F704E026B6033E402E435660A6
S2140110C041E01E0042695768364D3D40F6B237048E
S2140110D0E026F6023E402E43566034E00226426980
S2140110E05768304D3D40F6B23704E026F6023E40E2
S2140110F02E43566027E0032642695768294D3D4036
S214011100F6B23704E026F6023E402E4356601AE059
S214011110042642695768234D3D40F6B23704E0265F
S214011120F6023E402E4356600DE00526426957689A
S2140111301C4D3D40F6B23704E026F6023E402E43F3
S214011140566000E021000A00D2B2002A17D0009AA9
S2140111509288002A12D0009A9288092A0EDA009AFA
S2140111609688761E426957686D4D3D40F6B2370245
S214011170E026F6003E402E43566000E02100009A2D
S2140111801278002A00D12300406942681024A24345
S214011190DBB21B0110242340134343600800C0B296
S2140111A0F2BD0000FFFFF8FFFFFFC7FF006A0860FF
S2140111B00120704700B54068806C02091000C00726
S2140111C0C00FC0B2002804D0FA20800008600120B9
S2140111D000E0002000BD00B50978002901D00121FA
S2140111E000E000214068826C10239A43C9B20901CD
S2140111F01023194011438164012000BD00B54068E9
S214011200406C02091000C007C00FC0B2002804D00D
S214011210FA20C0010860012000E0002000BD00B5F2
S2140112200978002901D0012100E000214068426CC4
S21401123010239A43C9B2090110231940114341648E
S214011240012000BDFA20400208600120704710B559
S2140112500200002054680123646824091C40E4B29B
S214011260002C01D1002015E054686468240C1C4051
S214011270E4B2002C03D11000FFF775FC09E05468B6
S2140112806468240C2340DBB2012B02D1100000F06D
S21401129009F9C0B210BDF3B500221100160043686B
S2140112A05F681024E44327401025F6B236012E402D
S2140112B03E435E60019B5B780A2B0DD116004368A6
S2140112C05F6818493940F6B2360480277F023E40EF
S2140112D00E435E60012112E0019B5B78182B0ED154
S2140112E0012143685F680F4E3E400096009EC9B2DA
S2140112F0090480277F023940314359600121019B4F
S2140113001B78002B01D00122FFE7406843681C4090
S214011310D2B212011540254345600800C0B2F6BDA1
S214011320FFF8FFFFFFFFFEFF10B50A00002143682C
S2140113309B681C092300DB07DB0FDBB2002B03D005
S2140113401100FFF742FC01000800C0B210BD00B555
S2140113500978002901D0012100E000214068826857
S21401136010239A43C9B20901102319401143816021
S214011370012000BD10B50A0000214368DB681C0986
S2140113802300DB07DB0FDBB2002B03D01100FFF7D6
S2140113901CFC01000800C0B210BD00B50978002988
S2140113A001D0012100E000214068C26810239A4361
S2140113B0C9B20901102319401143C160012000BDC3
S2140113C010B50A00002143681B691C092300DB07CE
S2140113D0DB0FDBB2002B03D01100FFF7F6FB010099
S2140113E00800C0B210BD00B50978002901D001215E
S2140113F000E000214068026910239A43C9B209013E
S2140114001023194011430161012000BD10B50A00E7
S214011410002143685B691C092300DB07DB0FDBB295
S214011420002B03D01100FFF7D0FB01000800C0B26B
S21401143010BD00B50978002901D0012100E0002186
S2140114404068426910239A43C9B209011023194022
S21401145011434161012000BD10B50A000021436817
S2140114609B691C092300DB07DB0FDBB2002B03D0D3
S2140114701100FFF7AAFB01000800C0B210BD00B5BD
S2140114800978002901D0012100E000214068826925
S21401149010239A43C9B209011023194011438161EF
S2140114A0012000BDF8B504000D00002007000090E3
S2140114B06068C06901090800C007C00FC0B20028F3
S2140114C001D1002054E060680726C069000C304056
S2140114D0C0B200280BD0022815D00ED304281ED087
S2140114E017D3062827D020D307282AD02FE069460D
S2140114F02000FFF7BFF8070029E069462000FEF745
S214011500A5FF070023E069462000FFF7C4F907009E
S2140115101DE069462000FFF795FE070017E06946C3
S2140115202000FFF747FE070011E069462000FFF79D
S21401153065FE07000BE069462000FFF737FE07004F
S21401154005E069462000FFF795F80700FFE7380039
S214011550C0B200280AD06068C069000A064031009F
S214011560C9B2491C009801F08CFB28603800C0B253
S214011570F2BDF2B501231900002426004568EA6988
S2140115801027BA43F6B2360110273E401643EE61E5
S214011590009A5278032A19D0052A0AD0072A22D09F
S2140115A00E2A54D00F2A38D0102A43D0112A27D019
S2140115B05AE026004268D769CC4D3D40F6B2370462
S2140115C0E026F6023E402E43D6614EE01E004268FB
S2140115D0D769C64D3D40F6B23704E026F6023E40D6
S2140115E02E43D66141E002264268D769BF4D3D4091
S2140115F0F6B23704E026F6023E402E43D66134E0CA
S21401160003264268D769B94D3D40F6B23704E02655
S214011610F6023E402E43D66127E004264268D7698B
S214011620B24D3D40F6B23704E026F6023E402E4368
S214011630D6611AE005264268D769AC4D3D40F6B240
S2140116403704E026F6023E402E43D6610DE006261C
S2140116504268D769A54D3D40F6B23704E026F6024A
S2140116603E402E43D66100E02100009A9288002A6F
S21401167012D0009A9288092A0EDA009A9688761E67
S2140116804268D769BA4D3D40F6B23702E026F60009
S2140116903E402E43D66100E02100009A1278002ACF
S2140116A000D123004068C2691024A243DBB21B01AB
S2140116B0102423401343C3610800C0B2F2BD10B525
S2140116C00200002054680123246A24091C40E4B265
S2140116D0002C01D100201FE05468246A240CA407C2
S2140116E0A40FE4B2002C05D0022C0BD006D3032C99
S2140116F00CD010E01000FEF7BDFF0CE01000FFF765
S214011700CAF808E01000FEF7A1FE04E0FA20400245
S21401171008601800FFE7C0B210BDF3B501210A004A
S2140117206B461A70002216004468256A10239D43F2
S2140117301023F6B236011E402E432662019C6478C1
S214011740032C20D0052C04D0072C0FD0112C27D029
S21401175033E016004468276AC54D3D40F6B23704AB
S214011760C026B6023E402E43266228E00E0044689C
S214011770276ABF4D3D40F6B23704C026B6023E404A
S2140117802E4326621BE002264468276AB84D3D4078
S214011790F6B23704C026B6023E402E4326620EE05D
S2140117A003264468276AB24D3D40F6B23704C02688
S2140117B0B6023E402E43266201E06C462270019C32
S2140117C02478002C00D111004068026A1024A2433C
S2140117D0C9B209010B401343036268460078F6BD9F
S2140117E010B50200002053689B6A1C092300DB0722
S2140117F0DB0FDBB2002B01D100201EE053689B6A91
S2140118001B0C9B079B0FDBB2002B05D0022B0BD0CA
S21401181006D3032B0CD00FE01000FFF7EFFC0BE014
S2140118201000FFF7C3FC07E01000FFF7C3FC03E05E
S2140118301000FFF7BFFCFFE7C0B210BDF3B50022F2
S2140118401100160043689F6A1024E44327401025C0
S214011850F6B236012E403E439E62019B5B78102B0A
S2140118600DD1160041688F6A814B3B40F6B23704B2
S214011870C026B6023E401E438E62012124E0019B33
S2140118805B780E2B0FD1012143689F6A784E3E404C
S2140118900096009EC9B20F04C02189023940314327
S2140118A09962012110E0019B5B780F2B0CD1022677
S2140118B041688F6A6E4B3B40F6B23704C026B602CB
S2140118C03E401E438E620121019B1B78002B01D0F6
S2140118D00122FFE74068836A1C40D2B2120115401C
S2140118E0254385620800C0B2F6BD0000FFFFF8FF81
S2140118F010B50200002054680123246B240C1C4000
S214011900E4B2002C03D11000FFF75FF909E0546838
S214011910246B240C2340DBB2012B02D11000FFF70D
S21401192091FCC0B210BD10B50200002318004C781F
S2140119300B2C0BD151680A6B8D4C1440DBB21A0488
S21401194080235B021A4022430A630EE0497811297C
S2140119500BD101215268136B854C1C40C9B2090496
S21401196080235B02194021431163C0B210BD000001
S214011970FFF8FFFF10B50200002054680123646BD6
S214011980240C1C40E4B2002C03D11000FFF71DF913
S21401199009E05468646B240C2340DBB2012B02D1AE
S2140119A01000FFF74FFCC0B210BD10B502000023B7
S2140119B018004C780B2C0BD151684A6B6C4C1440B8
S2140119C0DBB21A0480235B021A4022434A630EE00C
S2140119D0497811290BD101215268536B644C1C4084
S2140119E0C9B2090480235B02194021435163C0B286
S2140119F010BD10B50200002054680123A46B240C0E
S214011A001C40E4B2002C03D11000FFF7DEF809E019
S214011A105468A46B240C2340DBB2012B02D11000C6
S214011A20FFF710FCC0B210BD10B50200002318006D
S214011A304C780B2C0BD151688A6B4D4C1440DBB2A1
S214011A401A0480235B021A4022438A630EE0497817
S214011A5011290BD101215268936B454C1C40C9B228
S214011A60090480235B02194021439163C0B210BD73
S214011A70FFFFFCFF10B50200002054680123E46B51
S214011A80240C1C40E4B2002C03D11000FFF79DF893
S214011A9009E05468E46B240C2340DBB2012B02D12D
S214011AA01000FFF7CFFBC0B210BD10B50200002337
S214011AB018004C780B2C0BD15168CA6B2C4C144077
S214011AC0DBB21A0480235B021A402243CA630EE08B
S214011AD0497811290BD101215268D36B244C1C4043
S214011AE0C9B2090480235B0219402143D163C0B205
S214011AF010BD10B50200002054680123246C240C8C
S214011B001C40E4B2002C03D11000FFF75EF809E098
S214011B105468246C240C2340DBB2012B02D1100044
S214011B20FFF790FBC0B210BD10B5020000231800ED
S214011B304C780B2C0BD151680A6C0D4C1440DBB25F
S214011B401A0480235B021A4022430A640EE0497895
S214011B5011290BD101215268136C054C1C40C9B2E6
S214011B60090480235B02194021431164C0B210BDF1
S214011B70FFFFFEFF10B50200002014680123E46891
S214011B8024091C40E4B2002C03D11000FFF71DF815
S214011B900AE01268D26812091A40D2B2012A03D1A9
S214011BA0FA20400208601800C0B210BD10B502004D
S214011BB0002318004C780B2C0BD11068C16810223A
S214011BC09143DBB21A0110231A400A43C260012076
S214011BD00EE0497811290BD1012001001268D36863
S214011BE01024A343C9B20901102421401943D1602E
S214011BF0C0B210BD80B50269126813091A00D20777
S214011C00D20FD2B2002A01D1002001E0FEF7ABFFCD
S214011C1002BD00B50978002901D0012100E00021AC
S214011C200069026810239A43C9B2090110231940BA
S214011C3011430160012000BD80B502695268130995
S214011C401A00D207D20FD2B2002A01D1002001E039
S214011C50FEF7BBFF02BD00B50978002901D00121BE
S214011C6000E000210069426810239A43C9B20901C5
S214011C701023194011434160012000BD80B502695F
S214011C80126913091A00D207D20FD2B2002A01D163
S214011C90002001E0FEF799FF02BD00B50978002992
S214011CA001D0012100E000210069026910239A4356
S214011CB0C9B209011023194011430161012000BD79
S214011CC080B50269526913091A00D207D20FD2B23F
S214011CD0002A01D1002001E0FEF777FF02BD00B522
S214011CE00978002901D0012100E00021006942693C
S214011CF010239A43C9B209011023194011434161C7
S214011D00012000BD80B50269926913091A00D20745
S214011D10D20FD2B2002A01D1002001E0FEF723FF44
S214011D2002BD00B50978002901D0012100E000219B
S214011D300069826910239A43C9B209011023194028
S214011D4011438161012000BD80B50269D269130982
S214011D501A00D207D20FD2B2002A01D1002001E028
S214011D60FEF733FF02BD00B50978002901D0012135
S214011D7000E000210069C26910239A43C9B2090133
S214011D80102319401143C161012000BDF8B50400BC
S214011D900E0020690125006A010928000840C0B22A
S214011DA0002801D1002035E028000027009720698F
S214011DB0006A000C8007800FC0B2002805D00228F8
S214011DC00FD008D3032812D017E069462000FEF78B
S214011DD003FA070011E069462000FEF791F90700B3
S214011DE00BE069462000FEF707FA070005E06946A2
S214011DF02000FEF7F1F90700FFE72069006A000AF4
S214011E008007800F85402900009800F03AFF306077
S214011E103800C0B2F2BDFCB500231A001F000669E7
S214011E20356A1024A5431024FFB23F0127402F43F3
S214011E3037624D78012D01D11D000AE04D78002D45
S214011E4001D1012505E04D78022D01D1022500E0E2
S214011E50FF252E00F6B2FF2E0BD00269176AA24E9E
S214011E603E40EDB22F04C025AD023D40354315621C
S214011E7001221500EDB2002D2CD08D88012D01D147
S214011E801D000FE08D88022D01D101250AE08D8805
S214011E90042D01D1022505E08D88082D01D10325E9
S214011EA000E0FF252E00F6B2FF2E12D06E463570EA
S214011EB005692F6A8D4E3E400196019FBC466E46CF
S214011EC036783702C026B6003E4067463E432E624D
S214011ED000E01A000978002901D00123FFE7006914
S214011EE0016A1025A943DBB21B011C400C430462A6
S214011EF01000C0B2F6BD80B50269926A13091A00D5
S214011F00D207D20FD2B2002A01D1002001E0FEF79B
S214011F105CFE02BD00B50978002901D0012100E070
S214011F2000210069826A10239A43C9B2090110236D
S214011F30194011438162012000BD80B50369012269
S214011F401B6B1B091340DBB2002B01D100201BE0E9
S214011F500269126B120C9207920FD2B2002A05D0B8
S214011F60022A09D005D3032A09D00BE0FEF782FB2B
S214011F7009E0FEF76BFA06E0FEF78DFC03E0FEF7DC
S214011F8079FB00E00020C0B202BDF2B500221100CC
S214011F90160003691F6B1024E44327401025F6B290
S214011FA036012E403E431E63009B5B78052B01D114
S214011FB013000CE0009B5B78032B01D1012306E0A4
S214011FC0009B5B78072B01D1022300E0FF231E0054
S214011FD0F6B2FF2E0BD001690F6B434E3E40DBB2CB
S214011FE01F04C0239B023B4033430B630121009B2C
S214011FF01B78002B01D00122FFE70069036B1C4010
S214012000D2B212011540254305630800C0B2F2BDE5
S21401201080B5036901225B6B1B091340DBB2002B01
S21401202001D100201BE00269526B120C9207920F3D
S214012030D2B2002A05D0022A09D005D3032A09D034
S2140120400BE0FEF717FB09E0FEF700FA06E0FEF7E5
S21401205022FC03E0FEF70EFB00E00020C0B202BD4A
S214012060F2B500221100160003695F6B1024E443E9
S21401207027401025F6B236012E403E435E63009B94
S2140120805B78052B01D113000CE0009B5B78032BDA
S21401209001D1012306E0009B5B78072B01D10223C7
S2140120A000E0FF231E00F6B2FF2E0BD001694F6B36
S2140120B00D4E3E40DBB21F04C0239B023B40334320
S2140120C04B630121009B1B78002B01D00122FFE707
S2140120D00069436B1C40D2B212011540254345638B
S2140120E00800C0B2F2BD0000FFFFFCFFFFFCFFFFCF
S2140120F080B5036901221B6C1B091340DBB2002B60
S21401210001D100201BE00269126C120C9207920F9B
S214012110D2B2002A05D0022A09D005D3032A09D053
S2140121200BE0FEF7A7FA09E0FEF790F906E0FEF7E6
S214012130B2FB03E0FEF79EFA00E00020C0B202BD4B
S214012140F2B500221100160003691F6C1024E44347
S21401215027401025F6B236012E403E431E64009BF2
S2140121605B78052B01D113000CE0009B5B78032BF9
S21401217001D1012306E0009B5B78072B01D10223E6
S21401218000E0FF231E00F6B2FF2E0BD001690F6C94
S214012190AD4E3E40DBB21F04C0239B023B4033439F
S2140121A00B640121009B1B78002B01D00122FFE765
S2140121B00069036C1C40D2B2120115402543056428
S2140121C00800C0B2F2BD80B5036901225B6C1B0931
S2140121D01340DBB2002B01D100201BE00269526CD8
S2140121E0120C9207920FD2B2002A05D0022A09D009
S2140121F005D3032A09D00BE0FEF73CFA09E0FEF707
S21401220025F906E0FEF747FB03E0FEF733FA00E0A8
S2140122100020C0B202BDF2B500221100160003690B
S2140122205F6C1024E44327401025F6B236012E4099
S2140122303E435E64009B5B78052B01D113000CE0E6
S214012240009B5B78032B01D1012306E0009B5B78A2
S214012250072B01D1022300E0FF231E00F6B2FF2E5A
S2140122600BD001694F6C784E3E40DBB21F04C02391
S2140122709B023B4033434B640121009B1B78002BA0
S21401228001D00122FFE70069436C1C40D2B2120163
S2140122901540254345640800C0B2F2BD80B5036908
S2140122A001229B6C1B091340DBB2002B01D10020DD
S2140122B01BE00269926C120C9207920FD2B2002AAE
S2140122C005D0022A09D005D3032A09D00BE0FEF770
S2140122D0D1F909E0FEF7BAF806E0FEF7DCFA03E00A
S2140122E0FEF7C8F900E00020C0B202BDF2B5002238
S2140122F01100160003699F6C1024E4432740102543
S214012300F6B236012E403E439E64009B5B78052B59
S21401231001D113000CE0009B5B78032B01D1012354
S21401232006E0009B5B78072B01D1022300E0FF2328
S2140123301E00F6B2FF2E0BD001698F6C974E3E4001
S214012340DBB21F04C0239B023B4033438B64012155
S214012350009B1B78002B01D00122FFE70069836CEC
S2140123601C40D2B212011540254385640800C0B254
S214012370F2BD80B5036901221B6E1B091340DBB257
S214012380002B01D100201BE00269126E120C92078D
S214012390920FD2B2002A05D0022A09D005D3032A09
S2140123A009D00BE0FEF766F909E0FEF74FF806E004
S2140123B0FEF771FA03E0FEF75DF900E00020C0B217
S2140123C002BDF2B500221100160003691F6E10242B
S2140123D0E44327401025F6B236012E403E431E66E2
S2140123E0009B5B78052B01D113000CE0009B5B780A
S2140123F0032B01D1012306E0009B5B78072B01D15B
S214012400022300E0FF231E00F6B2FF2E0BD0016967
S2140124100F6E624E3E40DBB21F04C0239B023B4060
S21401242033430B660121009B1B78002B01D0012250
S214012430FFE70069036E1C40D2B212011540254326
S21401244005660800C0B2F2BDFFFFFCFF7CB50500C3
S2140124500C0029690120496E0A0901001140C9B220
S214012460002901D1002037E0002600962869406E39
S214012470000C8007800FC0B2002805D002280FD0BC
S21401248008D3032812D017E069462800FDF7A4FEFA
S214012490060011E069462800FDF732FE06000BE053
S2140124A069462800FDF7A8FE060005E069462800F3
S2140124B0FDF792FE0600FFE72869406E000A8106D6
S2140124C0890EC9B2491C022900D20221009800F0E7
S2140124D0D8FB20603000C0B276BDF3B50100002203
S2140124E0100016000C69656E10239D431023F6B28A
S2140124F036011E402E436666019C6478012C01D18C
S21401250014000CE0019C6478002C01D1012406E043
S214012510019C6478022C01D1022400E0FF242500EE
S214012520EDB2FF2D0BD00869466E1C4D3540E4B266
S2140125302604C024A40234402C434466012004002F
S214012540E4B2002C18D0019CA488A41E3F2C12D201
S214012550019CA5886D1E0C69666E0096009F104E44
S2140125603E400096009EEDB22F02FC25AD013D4097
S2140125703543656600E01000019C2478002C01D0EC
S2140125800122FFE709694C6E1025AC43D2B2120155
S214012590134023434B66C0B2F6BD0000FFFFFCFFAD
S2140125A0FFC0FFFF0020704700B50978002901D061
S2140125B0012100E000210069826E10239A43C9B20E
S2140125C009011023194011438166012000BD80B521
S2140125D00269D26E13091A00D207D20FD2B2002AAC
S2140125E001D1002001E0FEF7F0FA02BD00B509783E
S2140125F0002901D0012100E000210069C26E1023EC
S2140126009A43C9B20901102319401143C16601203A
S21401261000BD80B50269126F13091A00D207D20FE6
S214012620D2B2002A01D1002001E0FEF7CEFA02BDA7
S21401263000B50978002901D0012100E000210069D8
S214012640026F10239A43C9B209011023194011439E
S2140126500167012000BD80B502698023D2581309A5
S2140126601A00D207D20FD2B2002A01D1002001E00F
S214012670FEF779FA02BD00B50978002901D00121DB
S21401268000E0002100698022825810239A43C9B2D3
S214012690090110231940114380228150012000BDF9
S2140126A080B502698423D25813091A00D207D20FC3
S2140126B0D2B2002A01D1002001E0FEF754FA02BD91
S2140126C000B50978002901D0012100E00021006948
S2140126D08422825810239A43C9B209011023194053
S2140126E0114384228150012000BD80B502699423E4
S2140126F0D25813091A00D207D20FD2B2002A01D13A
S214012700002001E0FDF7FCFC02BD00B509780029B8
S21401271001D0012100E00021006994228258102393
S2140127209A43C9B2090110231940114394228150DA
S214012730012000BD80B502699C23D25813091A00F6
S214012740D207D20FD2B2002A01D1002001E0FDF754
S21401275053FD02BD00B50978002901D0012100E032
S214012760002100699C22825810239A43C9B20901AC
S2140127701023194011439C228150012000BD406A5C
S214012780086001207047806A086001207047C06AAF
S21401279008600120704780B501220269A023D25843
S2140127A0120C5207520FD2B2002A0BD0022A0FD0B7
S2140127B00BD3042A12D00ED3062A15D011D3072A1A
S2140127C012D014E0FFF7DBFF12E0FFF7DCFF0FE0AB
S2140127D0FFF7DDFF0CE0FDF7D7FF09E0FDF7BDFED3
S2140127E006E0FEF7DFF803E0FDF7CEFF00E000208D
S2140127F0C0B202BD10B502000123180049780429B1
S21401280045D0062934D0082950D0372904D0382994
S21401281011D039291DD058E000231169A0228A5809
S214012820BA4C1440DBB21B04E022D2021A40224307
S214012830A023CA504AE01169A0228A58B34C14401A
S214012840DBB21B04E022D2021A402243A023CA5064
S2140128503CE002231169A0228A58AC4C1440DBB23A
S2140128601B04E022D2021A402243A023CA502DE0C4
S21401287003231169A0228A58A44C1440DBB21B041E
S214012880E022D2021A402243A023CA501EE00423AB
S2140128901169A0228A589D4C1440DBB21B04E02229
S2140128A0D2021A402243A023CA500FE00523116921
S2140128B0A0228A58954C1440DBB21B04E022D202B7
S2140128C01A402243A023CA5000E00020C0B210BD27
S2140128D080B501220269A423D258120C5207520F66
S2140128E0D2B2002A0BD0022A0FD00BD3042A12D060
S2140128F00ED3062A15D011D3072A12D014E0FFF7FB
S2140129003EFF12E0FFF73FFF0FE0FFF740FF0CE04E
S214012910FDF73AFF09E0FDF720FE06E0FEF742F874
S21401292003E0FDF731FF00E00020C0B202BD10B5A4
S2140129300200012318004978042945D0062934D01D
S214012940082950D0372904D0382911D039291DD06B
S21401295058E000231169A4228A586C4C1440DBB25B
S2140129601B04E022D2021A402243A423CA504AE0A2
S2140129701169A4228A58654C1440DBB21B04E0227C
S214012980D2021A402243A423CA503CE00223116912
S214012990A4228A585D4C1440DBB21B04E022D2020A
S2140129A01A402243A423CA502DE003231169A4220E
S2140129B08A58564C1440DBB21B04E022D2021A405D
S2140129C02243A423CA501EE004231169A4228A5874
S2140129D04E4C1440DBB21B04E022D2021A402243C2
S2140129E0A423CA500FE005231169A4228A58474C34
S2140129F01440DBB21B04E022D2021A402243A42375
S214012A00CA5000E00020C0B210BD10B501231A0064
S214012A100269C0241259120C1340DBB2002B02D0FB
S214012A20012B03D005E0FEF7E9FB03E0FEF7BEFB52
S214012A3000E00020C0B210BD10B50200012318004E
S214012A4049780E2910D010291CD100231169C02203
S214012A508A587A4C1440DBB21A0480235B021A406F
S214012A602243C023CA500EE01169C0228A58734C13
S214012A701440DBB21A0480235B021A402243C023AF
S214012A80CA5000E00020C0B210BD10B501231A00E4
S214012A900269C4241259120C1340DBB2002B02D077
S214012AA0012B03D005E0FEF7A9FB03E0FEF77EFB52
S214012AB000E00020C0B210BD10B5020001231800CE
S214012AC049780E2910D010291CD100231169C4227F
S214012AD08A585A4C1440DBB21A0480235B021A400F
S214012AE02243C423CA500EE01169C4228A58534CAB
S214012AF01440DBB21A0480235B021A402243C4232B
S214012B00CA5000E00020C0B210BD0000FFFFF8FF71
S214012B1080B50269CC23D25813091A00D207D20F06
S214012B20D2B2002A01D1002001E0FEF71CF802BD56
S214012B3000B50978002901D0012100E000210069D3
S214012B40CC22825810239A43C9B209011023194096
S214012B501143CC228150012000BDF0B5059D069E93
S214012B60079F089C016042608360C56006614761FB
S214012B70216881616168C161A168016200210A0062
S214012B800AE00A00D2B29200A218D2680B00DBB2A9
S214012B909B00C3185A62491C0A00D2B2032AF0D31A
S214012BA0F0BD38B503000C0011002000C0B23F286C
S214012BB001DB00200DE00020214A2500EDB2ED00EA
S214012BC05559002D04D01800E4B2E300D2589047BE
S214012BD0C0B232BDF8B50B0015001900C9B23F29C5
S214012BE001DB002029E000242100154A1E00F6B270
S214012BF0F60096197668002E1DD0290005001148AA
S214012C006F688026B8511048AE6830660F482F6846
S214012C108026B8512800DBB2DB00D21852689047F4
S214012C20010020006A688023D0502000AA68106640
S214012C302868802284500800C0B2F2BDFFFFFEFF64
S214012C402C97010052455355202096194B4D43525F
S214012C50F446002804D4494200F013F84042604785
S214012C604042002905D45FD000F00BF840424942AB
S214012C706047494200F005F84942604703460B4366
S214012C80E6D40022030A8B420BD203098B4219D2E7
S214012C9043088B422ED2411A00D2014652411046B9
S214012CA07047FF2209023FD012068B4205D312124B
S214012CB009028B4201D31212090203098B4219D36E
S214012CC000E0090AC3098B4201D3CB01C01A524165
S214012CD083098B4201D38B01C01A524143098B42AF
S214012CE001D34B01C01A524103098B4201D30B0198
S214012CF0C01A5241C3088B4201D3CB00C01A5241BD
S214012D0083088B4201D38B00C01A524143088B4281
S214012D1001D34B00C01A5241884200D3401A524197
S214012D20CFD201461046704708B500F001F808BD3D
S214012D307047010000B501000020C9B2002905D086
S214012D40022907D004D3032906D006E0102004E0A8
S214012D50182002E0282000E04820C0B200BD70B56F
S214012D600E0001680C008034002529002900006847
S214012D70C9B2002919D0022909D00FD303291BD1C2
S214012D80C02109014058400E8507AD0F14E0C0214F
S214012D9009014058800D8507AD0F0DE0C0210901DE
S214012DA04058C00C8507AD0F06E0C0210901405808
S214012DB0000C8507AD0FFFE72800C0B2FFF7BAFF8A
S214012DC00100C9B2890830002A00D2B2002A05D112
S214012DD0C9B280B241438800201832E02A00D2B23C
S214012DE0012A0ED1C9B2020092B251430D0080B23F
S214012DF01521FFF743FF400029000818800020181E
S214012E001FE0EDB2022D0ED1C9B2020092B25143BB
S214012E100D0080B20C21FFF731FFC0002900081811
S214012E20800020180DE0C9B2020092B251430D0095
S214012E3080B20721FFF722FF400029000818800012
S214012E40201870BD00B5010000200A00D2B2002A89
S214012E50082A0ED9093A0ED0521E0ED0521E0ED096
S214012E60521E0ED0521E0ED0521E0ED0521E0ED024
S214012E700FE008000DE00C200BE0102009E0142004
S214012E8007E0182005E0202003E0302001E0402084
S214012E90FFE7C0B200BD80B500231A0089B2FFF774
S214012EA05EFF0068000C0007000FC0B2FFF7CAFF04
S214012EB0C0B202BD00B50023D2B2002A0CD002680F
S214012EC0C023DB03134303604268520F5207C90055
S214012ED0C908114341600BE00268B14B134003601F
S214012EE04268B04B13408A04AF4911401943416010
S214012EF000BD0268AD4B134003600268C9B2090405
S214012F00F0231B030B4013430360704700B50268B0
S214012F105200520802600268A54B13400360C9B212
S214012F20002909D00168802212060A43026001685E
S214012F308022D2050A43026000BD00B50A00D2B263
S214012F40002A06D101689B4A0A40026001680160B6
S214012F500BE0C9B2012908D10168964A0A4002600D
S214012F6001688022D2040A43026000BD10B50168E0
S214012F70803100221300140003E0A300CB181A606E
S214012F80641C037EDB019C42F7D310BD10B48A4952
S214012F9082688023D15001214268136D2024A34307
S214012FA0C9B24901202421401943116500218068D6
S214012FB08022815010BC704710B47F4982688023FC
S214012FC0D15001214268136D1024A343C9B20901EF
S214012FD01024214019431165002180688022815008
S214012FE010BC7047F0B4049C059D069E079F3F7871
S214012FF00776016042608360C46005614661F0BC8B
S214013000704710B500210A0081600161416181614C
S214013010C160C16141628162C162016201220270C6
S2140130200A00C2700A0002710022D2434263826320
S214013030C26302640B00442403550B004524035568
S2140130400B00C82403550823462403550B0005E04E
S2140130501C00E4B2A4000419A2645B1C1C00E4B2C8
S214013060202CF5DB0A0042700A0082700A00302329
S214013070C2540A00C923C2540A00CA23C2540A0011
S214013080CB23C2540A00D523C2540A00D423C25407
S2140130900A00D623C2540A00D723C2540A00CC23FE
S2140130A0C254D022815010BD30B500210A000368F9
S2140130B01C683F4D2540D2B292078024E405224089
S2140130C02A431A60026813683C4C1C40C9B20907BF
S2140130D080235B05194021431160016809680A0EC7
S2140130E01100C907C90FC9B20029F6D130BD38B5DC
S2140130F00400206801250068000D2840C0B20028A1
S21401310013D0002021680A6852005208C0B2C007D6
S2140131101043086002E02000FFF74EFF20680068B9
S214013120000D2840C0B20028F5D1280021680A68A1
S214013130234B1340C0B2400680229204104018432D
S214013140086020680068400E2840C0B20028F8D108
S214013150280021680A68164B1340C0B280078022F7
S214013160D205104018430860280021680A68134BEE
S2140131701340C0B200078022520510401843086071
S21401318020680068000E2840C0B20028F8D02068E9
S2140131900068C00E2840C0B20028F1D031BD000042
S2140131A0FFFF9FFFFFFF03E00000FC1FFFFFF0FF94
S2140131B0FFFFFFBFFFFFFFF052455355FFFFFFEF35
S2140131C0FFFFFFFDF0B593B007000C0015002900C6
S2140131D0C9B289B23800FFF7C2FD0600227A6168DB
S2140131E03000FFF767FEA17A3000FFF782FEE17A32
S2140131F03000FFF78BFE617A3000FFF79EFE207BE2
S214013200002805D0684605706946380000F0A8FD1C
S214013210607A012807D120693968EDB2AA008918B9
S21401322088221201885013B0F0BD0000F8B50400E2
S2140132300E00002500202000FFF7A8FE0127390018
S2140132402068026852005208C9B2C90711430160DA
S21401325020680068010D38000840C0B20028F7D089
S214013260327821684B686D481840D2B252038023E9
S2140132709B011A4002434A602000FFF738FF3A00DC
S21401328021680B6866481840D2B2D20580231B0419
S2140132901A4002430A603A0021684B6B61481840A5
S2140132A0D2B2120780235B051A4002434A6320000C
S2140132B0FFF75CFE3020305CFFF73CFD01000800A4
S2140132C0C0B2002807D080208000C9B2FFF7D9FC21
S2140132D00500207E4543206801687F229143EDB2B8
S2140132E06A06520E0A430260380021680A6D5200CF
S2140132F05208C0B2C007104308654B49B06843186E
S2140133002068056D494A2A409BB25D05484B2B4013
S21401331013430365F06843182068056D454A2A4043
S2140133201D04F8235B032B401343036530694318E0
S2140133302068056D404A2A409BB29D02FC231B0271
S2140133402B4013430365706943182068056D3B4A9B
S2140133502A409BB25D01F8239B002B401343036573
S214013360B06943182068026D1F25AA439BB2DB068D
S214013370DB0E13430365F078002861D03B0022681A
S2140133801568D7482840DBB25B078025AD052B4082
S21401339003431360337922681568D2482840DBB2AC
S2140133A0DB0380252D022B4003431360306C22681B
S2140133B090644420335C20680568CB4A2A40DBB21F
S2140133C01D02C0239B002B40134303604520335C42
S2140133D02068456BC54A2A40DBB21D06F0231B0553
S2140133E02B4013434363C820305C012840D10022A0
S2140133F010004623F35CC0B2984239D21000C0B226
S21401340080003018836C15002068EDB2AD004519B8
S214013410882000012B50521CEAE700BFFFDFFFFFA8
S214013420FFFF7FFFFFFFFFEFFFFF0000FFFF1F8093
S2140134300000E07FFFFFE0FFFF03FFFF1FFCFFFF31
S214013440002322681568A6482840DBB25B07802562
S214013450AD052B4003431360002322681568A1487D
S2140134602840DBB2DB0380252D022B40034313608B
S2140134707078002800D16CE1737822681568CE4810
S2140134802840DBB2DB0280252D012B40034313606D
S2140134903A002068C0231B01C3585B005B08D2B208
S2140134A0D2071A43C0231B01C250F0694318226891
S2140134B0C2481558C24828409BB21D05C14B2B4037
S2140134C00343BE481350306A43182268BB48155858
S2140134D0BD4828401D04E023DB022B400343B748C8
S2140134E01350736A2268B5481558B84828409BB2ED
S2140134F09D02F823DB012B400343B0481350B06A0A
S21401350042182068AD4BC358E025AB4392B2550133
S214013510E0222A401A43A94BC250F06A411820689B
S214013520A64A825807239A4389B24907490F11438D
S214013530A24A81503020315C00232068C02212014B
S2140135408258DBB2002B1FD0022B0BD013D3032BD8
S21401355023D1C44B1340C9B24906C022D2040A4043
S2140135601A431AE0C04B1340C9B28905C02212049F
S2140135700A401A4311E0BD4B1340C9B2C904C02228
S21401358052030A401A4308E0B94B1340C9B2090472
S214013590C02292020A401A43FFE7C02109014250A5
S2140135A03020315C3B002068C02212018258DBB219
S2140135B0002B1FD0022B0BD013D3032B23D1A94BE7
S2140135C01340C9B24906C022D2040A401A431AE07F
S2140135D0A54B1340C9B28905C02212040A401A43FA
S2140135E011E0A24B1340C9B2C904C02252030A40DB
S2140135F01A4308E09E4B1340C9B20904C022920246
S2140136000A401A43FFE7C021090142503020315CCD
S21401361002232068C02212018258DBB2002B1FD081
S214013620022B0BD013D3032B23D18E4B1340C9B2DD
S2140136304906C022D2040A401A431AE08A4B1340B4
S214013640C9B28905C02212040A401A4311E0874B09
S2140136501340C9B2C904C02252030A401A4308E003
S214013660834B1340C9B20904C02292020A401A438E
S214013670FFE7C021090142503020315C0323206856
S214013680C02212018258DBB2002B1FD0022B0BD0B6
S21401369013D3032B2CD1734B1340C9B24906C02256
S2140136A0D2040A401A4323E06F4B1340C9B289057E
S2140136B0C02212040A401A431AE06C4B1340C9B2E6
S2140136C0C904C02252030A401A4311E0684B134052
S2140136D0C9B20904C02292020A401A4308E000BF98
S2140136E0FFFFFFDFFF7FFFFFFFFCFFFFFFFFFFF096
S2140136F0C02109014250CA20325C2068C02109015C
S2140137004358AA491940D2B2D20380231B021A4059
S2140137100A43C02109014250CB20325C2068C021F7
S21401372009014358A2491940D2B21302F8225201A4
S2140137301A400A43C02109014250B2782068436BFF
S2140137409C491940D2B2120380235B011A400A43F6
S2140137504263706B21680861B06B21684861F06B49
S21401376021688861C820325C206803689249194044
S214013770D2B2120480235B021A400A430260C920B7
S214013780305C002824D00022206803688B49194049
S214013790D2B2520480239B021A400A4302603A00C6
S2140137A02068436883491940D2B2120380235B0123
S2140137B01A400A43426023E0FFF7FFFF040C0000B3
S2140137C0FFFF0FC00000F03FFFFFF8FFFF83FFFF82
S2140137D03A002068036879491940D2B2520480231E
S2140137E09B021A400A43026000222068436871491E
S2140137F01940D2B2120380235B011A400A43426089
S214013800D420305C002835D03A00206803686C4923
S2140138101940D2B292058023DB031A400A430260A4
S2140138203A002068036867491940D2B2920680239D
S214013830DB041A400A4302603A00206803686249C2
S2140138401940D2B292048023DB021A400A43026076
S214013850380061698A6C01239A43C0B20740174356
S2140138608F6434E0FFFFFFF9FFFF3FFFFFFFE7FF35
S214013870FFFFFCFF00210B00226815685048284016
S214013880DBB29B058025ED032B40034313600B0041
S214013890226815684B482840DBB29B068025ED045C
S2140138A02B40034313600B002268156846482840E6
S2140138B0DBB29B048025ED022B4003431360606955
S2140138C0826C01239A43C9B20F4017438764D520FF
S2140138D0305C21680A68374B1340C0B2000380226F
S2140138E05201104018430860D620305C21684A68AF
S2140138F02E4B1340C0B2C003802212021040184360
S2140139004860D720305C21684A68304B1340C0B20B
S21401391080038022D201104018434860002723E02C
S2140139202A00D2B2D02030583900C9B214235943E4
S21401393041182000FFF746FC6D1C2A0092B2D020E9
S21401394030583900C9B214235943435AD02030584D
S21401395084463900C9B21420414360464018408865
S21401396018188242DCDB7F1C3800CC21715CC0B2A7
S214013970884208D20020D02030583900C9B214221B
S2140139805143455AD9E7200000F06EF92000FFF7B1
S2140139908BFB002021680A680D4B1340C0B2C0059E
S2140139A080221204104018430860F1BDFF7FFFFF1C
S2140139B0FFE0FFFFFFEFFFFFFFFFFEFFFFFFFDFF43
S2140139C0FFFFBFFFFFFFFFFBFFFFFBFFFFBFFFFF89
S2140139D0FFFF7FFF80B5097889B2FFF7C0F901685C
S2140139E0C02212050A43026001BDF8B506000C00AC
S2140139F0217889B23000FFF7B2F905000835217841
S214013A0089B23000FFF747FA00210A000A001BE0DE
S214013A101600F6B23340032B15D12B681600F6B20A
S214013A20A619367A1E432E602D1D0CE01600F6B23E
S214013A301E40022EECD12B681600F6B2A619367A75
S214013A4036021E432E60521C1300DBB283421BD289
S214013A5003231E00324209D129602B681600F6B2F4
S214013A60A619367A36061E432E60ECE71600F6B225
S214013A701E40012EDAD12B681600F6B2A619367A48
S214013A8036041E432E60DEE7F1BDF8B506000C00D5
S214013A90217889B23000FFF762F905002868000C2A
S214013AA00007000FFFF7CEF9482160542868400D43
S214013AB00100C907C90F281DC9B2002904D0016831
S214013AC0C900C908616004E00168890C4905490D0F
S214013AD06160051D217889B23000FFF7DCF900210D
S214013AE00A0012E02A680B00DBB2E3181A722D1DD9
S214013AF00AE00B00DBB21A40022AF3D12A68120A46
S214013B000B00DBB2E3181A72491C0A000300D2B29A
S214013B10DBB29A4216D203221300194206D12A6852
S214013B20120E0B00DBB2E3181A72EDE70B00DBB2E4
S214013B301340012BDDD12A68120C0B00DBB2E3180F
S214013B401A72E1E730688068F1BD30B500231A00CB
S214013B500A78D506ED0E01242200AA400D78402DE4
S214013B6011DB0221006800290AD0022904D005D3FE
S214013B70032907D1026705E0426703E0C26201E05C
S214013B800263FFE723E00978202910DB0068002C98
S214013B900AD0022C04D005D3032C07D1026705E016
S214013BA0426703E0C26201E00263FFE70FE00068DC
S214013BB0002B0AD0022B04D005D3032B07D10267B2
S214013BC005E0426703E0C26201E00263FFE730BD41
S214013BD030B5002213000B78DD06ED0E012423001C
S214013BE0AB400D78402D12DB0221006800290AD077
S214013BF0022904D005D3032907D1026F05E0426FDD
S214013C0003E0C26A01E0026BFFE71A4026E009788A
S214013C10202911DB0068002C0AD0022C04D005D321
S214013C20032C07D1026F05E0426F03E0C26A01E090
S214013C30026BFFE71A4011E01100006800290AD064
S214013C40022904D005D3032907D1026F05E0426F8C
S214013C5003E0C26A01E0026BFFE71A40002A01D0C6
S214013C60012000E0002030BD10B5017E032937D1C8
S214013C700021C9430A0002240368002C0AD0022C42
S214013C8004D005D3032C07D11A6705E05A6703E071
S214013C90DA6201E01A63FFE70A0001240368002CD8
S214013CA00AD0022C04D005D3032C07D11A6705E0ED
S214013CB05A6703E0DA6201E01A63FFE70022006850
S214013CC0002A0AD0022A04D005D3032A07D10167A5
S214013CD005E0416703E0C16201E00163FFE73EE002
S214013CE0017E022925D10021C9430A000124036867
S214013CF0002C0AD0022C04D005D3032C07D11A6756
S214013D0005E05A6703E0DA6201E01A63FFE7002282
S214013D100068002A0AD0022A04D005D3032A07D154
S214013D20016705E0416703E0C16201E00163FFE767
S214013D3015E0017E012912D10021C9430022006845
S214013D40002A0AD0022A04D005D3032A07D1016724
S214013D5005E0416703E0C16201E00163FFE710BDD2
S214013D6030B500231A000A78D506ED0E012422008C
S214013D70AA400D78402D19DB02210068002910D0D9
S214013D80022906D009D303290FD1816E0A43826620
S214013D900BE0C16E0A43C26607E0416A0A4342620B
S214013DA003E0816A0A438262FFE733E0097820294B
S214013DB018DB0068002C10D0022C06D009D3032C87
S214013DC00FD1816E0A4382660BE0C16E0A43C2665A
S214013DD007E0416A0A43426203E0816A0A4382625B
S214013DE0FFE717E00068002B10D0022B06D009D39E
S214013DF0032B0FD1816E0A4382660BE0C16E0A4324
S214013E00C26607E0416A0A43426203E0816A0A43E6
S214013E108262FFE730BDF9B58FB00D00179900201B
S214013E2001200490012003900820009003230293B0
S214013E30022414240C94784C0B94FA24A4050A94B6
S214013E40C9B2002909D1754909915E2608931F2137
S214013E507118491C0791069008E0704909912626B9
S214013E60089307217118491C079106900192019841
S214013E7000F0DEF8059001240D952EE0280000F0F4
S214013E80E7F80100380000F0EEF80700019800F0AE
S214013E90CFF80100380000F070F98021090400F025
S214013EA0C5F939D8019800F0C3F80100380000F0D0
S214013EB064F901000798A8420EDB059800F0B6F9F0
S214013EC00AD80494009505910C98A84204DB0800D2
S214013ED00B9900F0BFF927D3641C0998A04223DB95
S214013EE00D9800F0A5F80500200000F0B1F80100DB
S214013EF0280000F0B8F80700019800F099F80100D2
S214013F00380000F0B0F800F0B9F90500002D02D035
S214013F1006988542B2DA07E0019800F089F8390080
S214013F2000F02BF90100C5E710A80488200080B234
S214013F3000F07EF80A9900F0BEF905000098B0423C
S214013F4000DA009E0CE0380000F082F8290000F04C
S214013F5081F904D20296380000F07AF80500761E40
S214013F600898864216DB3000401C2D4948430099CC
S214013F70FEF784FE210089B2411A012903DB2100E4
S214013F8089B2471A02E0210089B20F1A210089B2CC
S214013F908842D8DA00980299401A401E0190214CB6
S214013FA00125169E1DE0310089B20F1A0CE01C484F
S214013FB068430099FEF762FE310089B2411A012971
S214013FC0F1DB310089B2471A380000F041F82100D0
S214013FD000F040F904D20395380000F039F80400E7
S214013FE06D1C0198A842E2DA0F9C049820600298A2
S214013FF000F0CAF90CA20CCA00F0D0F900F090FA51
S214014000A0600298A168401AE060019820610398B8
S214014010606011B0F0BD0000CDCCCC3DFF030000C8
S2140140201027000000401C46333333333333E33F5D
S2140140309D2102000AD002D4491E9218FCD5C9055A
S214014040100A1206524100D3012A48417047000067
S2140140509D210200EED55242F446FFF7EBFF012206
S214014060D2071043604730B405004D400122D20705
S21401407015404B180418240E25D01B0E2CD0FF2CEF
S21401408031D0FF2B34D0E41A000209021043114349
S21401409043084808D10D1B1A02D2641EDB181B18F0
S2140140A0DB18834200D31B1A4941F9D37F3423DD41
S2140140B0FF2C05DAE40548086041284330BC704708
S2140140C0FF20C005F9E728001B0E03D0FF2BF5D112
S2140140D04902F3D0D043F1E7FF2C01D14002F9D1D8
S2140140E0FF20C005E9E74002F4D1FF2BF8D1F1E744
S2140140F028004902E2D0EDE70B0200202442DCD181
S2140141005B129B1CD9D9D805D7E70122D207030039
S2140141104B402ED4431A01D2C01AC91830B44B18DA
S2140141200418240E1B0E22D0FF2C20D0E31A182BC5
S2140141301DDC09021143C40D641E0002104394469F
S2140141401925ED1A0A00AA40D940451801D36D0871
S214014150A41CE405D209280A2D062A436546AA416D
S214014160604103181B0EFF2B01D3C00DC00530BCE8
S2140141707047514006E05140CCE70122D2070300C8
S2140141804B40F8D4431A03D2C01AC91850405140C4
S21401419030B44B18090211430418240E1B0E40D0EC
S2140141A0FF2C3AD025009D410BD31ED8C50D4002E9
S2140141B0401A0BD3ED050100400AC905914168413B
S2140141C0D5E7C50D40024918401AD0D00121400854
S2140141D0491C0018FCD58C4204D36D1A000AED0563
S2140141E04019C4E7E8051040C1E7182DBFDCAC1C38
S2140141F00D00E140E5414D40012D4941C40D00024D
S2140142001043451A01D46D199543641EE405280A26
S2140142102D069541604130BC7047FF2BA7D1D8438E
S214014220A5E72442A3D10020A1E7FEE70CB40122B2
S21401423012060318DA4207D84B18DA4204D80200ED
S2140142400A43921802D281420CBC7047FCD08842C5
S2140142500CBC70470CB4012212060318DA4207D8C8
S2140142604B18DA4204D802000A43921802D2884256
S2140142700CBC7047FCD08142FAE7FEE70122D20768
S2140142800118090E7F3910D449421F310FD4001886
S21401429005D2C0011043C84000D5D0437047C001C5
S2140142A01043C84005D44042704700207047004282
S2140142B0F3D51000704730B405004D400122D207F7
S2140142C015404B180418240E2ED01B0E32D0FF2C8E
S2140142D034D0FF2B3AD0E4180002090210431143F0
S2140142E0000A090A9446C2B24A43000AC3B24B43C3
S2140142F0000A4843110A5B181A43D2B2190A091870
S21401430001D44918641E080A7F3C23DBFE2C08DA18
S214014310E40509061143634699416041284330BCD0
S2140143207047FF20C005F9E728001B0EFF2BF6D1CA
S214014330D043F4E72800FF2CF1D1F9E74002F7D18A
S214014340FF2B01D14902F3D1E005E7E7D805490281
S214014350E4D0EDE743020020641CDFD15B129B1C16
S214014360DCD9D805DAE7FEE7010042221201D21EA7
S214014370004207D002D4521E0018FCD5C10A4005DF
S21401438012058918704700000100EED54042F44638
S214014390FFF7EBFF0122D20711436047F0B50E008D
S2140143A05E400125ED072E40B446AE0ADF184C18D4
S2140143B0F44208D2F7420ED2640D01D07F0D12D11D
S2140143C000206146F0BD05D1F74201D87F0D05D129
S2140143D00020C143F0BDFBD1640DF9D00020C143DC
S2140143E0490549088FE0E419C902DB0229432B433A
S2140143F0DB0A460DC00231438E4630B487B295B211
S2140144007D432E0CADB2140C7C43A419260C240457
S21401441025439CB27C43A419190C7943270CC9196E
S214014420A4B20F043C43090C000C97B247432E0C70
S214014430BE193543ADB2170C4743360CBF19A6B2A9
S214014440BF193E043543240C3E0C36199FB2474330
S214014450BF19BCB23E0C89191F0C47437F183E0496
S2140144603443390C704680B297B247432E0CBE19BE
S2140144703543ADB2170C4743360CBF19A6B2BF1968
S2140144803E043543240C3E0C36199FB24743BF19F0
S214014490BCB23E0C89191F0C47437F183E043443B7
S2140144A0390C77463F0C90B278432E0C80190604DF
S2140144B0ADB22E43050CA0B22D18120C7A4350193A
S2140144C0020C80B2240CA4189AB27A43121914046E
S2140144D02043120C89181B0C7B43C91830BCEF0A09
S2140144E0394203D1B61940414941641E6F12BF0DCE
S2140144F0E41B0BDBFF19BC4211DA24050027420836
S214014500AE417841614166463143F0BD641C05D138
S214014510401C6141CF0201D34908F4E750E75DE74B
S2140145204A1812D2400DC90208430121C90708439F
S214014530520D40210901521A521C06D452421F3212
S21401454001D4D0407047C017704700207047FEE77F
S21401455000B50100C9B2802900DB7F20C0B200BDD2
S21401456000B50100C9B2F139092901D2012004E0E0
S2140145700100C9B2802900DB0020C0B200BDFEB533
S2140145800400002528006E463F2030703078F02762
S2140145900F430740377072701800C0B2FFF7D8FF9C
S2140145A0B070207800280FD0032003E00100C9B2C4
S2140145B07554401C0100C9B20829F7DB0822694678
S2140145C0E068A36D984704E003226946E068A36D9E
S2140145D0984740B2FEBD7CB50300002001000100F3
S2140145E069460F220A700A78DC8AF02525431540B1
S2140145F00D70020008E01C691500EDB2645D15003F
S214014600EDB24D196C70521C1400E4B2DD8AA4B2EE
S214014610AC42F0D31A78002A15D0020006E0140046
S214014620E4B2DD8A64190C196070521C1400E4B2FD
S2140146300725DE8AAD1BAC42F1DB08226946D86845
S2140146409B6D984706E0DA8A521CD2B26946D86852
S2140146509B6D984740B276BD1CB5040068461F2185
S21401466001700178E28A92B2120AF02313430B40DA
S2140146700370E18A417000210A00D2B2C9B208E093
S21401468022690B00DBB2D25C0B00DBB2C3189A7056
S214014690491C0A00D2B2062AF2DB08226946E06803
S2140146A0A36D9847010049B2002904D1218B891DC9
S2140146B021830121A17640B216BDFEB50400002576
S2140146C02800C0B268462F2101700178A27EF0232F
S2140146D013430B400370E18A228B8E1A310089B294
S2140146E0082900DB07262900C9B20AE02269238BC4
S2140146F00F00FFB2DB19D25C0B00DBB2C3185A7095
S214014700491C0A00D2B2330092B29BB29A42EDD350
S214014710217800291AD02900C9B22900C9B207E0B8
S2140147200A00D2B233009BB2D21882185570491CC7
S2140147300A00D2B207233700BFB2DB1B9A42EFDB77
S21401474008226946E068A36D984706E03200521CCD
S214014750D2B26946E068A36D9847010049B20029C4
S21401476009D1218B89192183A17E491CA176A17EBD
S214014770102900DBA57640B2FEBD70B5030000200F
S21401478004000F240D782600354205D0D2B2521E01
S2140147900D782540AA4208DA586D002802D09948BB
S2140147A0596D88470620C04315E00A781440422216
S2140147B09C5208E00200D2B28A185278DC6B0500DF
S2140147C0EDB26255401C0200D2B242241C5B92B28A
S2140147D0A242EFD3002070BD38B5030000200400CC
S2140147E0D2B2082A08D0586D002802D08648596DE2
S2140147F088470620C04339E00A781202F0242401D3
S21401480014404A78A2181400A4B2082C08DA586D8D
S214014810002802D07D48596D88470620C04325E010
S21401482040241C5B1500ADB2AC4208D2586D00287E
S21401483002D07748596D88470220C04316E04224CB
S2140148401A5308E00200D2B28A189278DC6B05008F
S214014850EDB26255401C0200D2B2062AF2DB0620F7
S21401486044215852012046215854002032BDF8B543
S2140148700300002528004620185C0C782407240F26
S214014880A04202D00320C0433EE04220185A4424EE
S2140148901C5B041B200080B2082800DB0724D2B270
S2140148A0521E200080B2824208DA586D002802D0DB
S2140148B05848596D88470620C04325E02A000BE07A
S2140148C0D86B1600F6B24427DF5BF6191700FFB265
S2140148D0CF197F788755521C1000C0B2260080B2CF
S2140148E0B6B2B042ECD34420185A001944215852AB
S2140148F04620185C401C462158544620185C102857
S21401490001DB46201D540020F2BD80B50100D2B265
S214014910032A08DA486D002802D03F48496D8847C7
S2140149200620C04300E0002002BD80B513009BB204
S2140149300A00C16800F001F802BDF8B504000025C0
S2140149402800002C02D10020C04359E0A08A19009B
S21401495089B2884208D2606D002802D0C048616DD5
S21401496088470220C0434BE03420205C012808D150
S214014970606D002802D0BB48616D88470120C043A6
S2140149803EE0E38228002083280007E00100C9B248
S214014990515C26690700FFB2F155401C0100C9B2FF
S2140149A01E0089B2B6B2B142F0D3E08A082804DA12
S2140149B02000FFF710FE060020E02000FFF74CFE67
S2140149C00600300040B2002818D12800A083280035
S2140149D0A0772800E077E06D80472200203203C2EE
S2140149E0083AE06D804700226430514122002832A7
S2140149F003C2083A2563012034216054300040B2D6
S214014A00F2BD0000D0AB0100FCAB010058AA0100CA
S214014A1090AA010028AC010048AC0100FEB51400C4
S214014A201A001300DBB29B1E072B00D317E10025EB
S214014A302B00DBB22B00DBB2029408E0029C1E00C6
S214014A40F6B2A45D6E461F00FFB2F4555B1C1C0057
S214014A501600E4B2F6B2B442F0D32B00DBB207E0A4
S214014A606C461E00F6B21700FFB2F619A5555B1C80
S214014A701C00E4B208261700FFB2F61BB442EFDBB7
S214014A806F4604000E003878C0B20009002806D030
S214014A90022858D01BD3032800D19DE0DFE0512027
S214014AA0205C012804D10520C0435021605401E058
S214014AB050202554D2B269462000FFF75EFE40B270
S214014AC0002803D1A663022051216054C7E051207B
S214014AD0205C012804D10520C0435021605401E028
S214014AE050202554D2B269462000FFF775FE01001A
S214014AF00222D24349B291420CD10720C043502131
S214014B006054512025540023002202212000FFF783
S214014B1036FDA4E040B2002814D1A663012051213D
S214014B20605460784721605401234720225C0021AD
S214014B302000FFF724FDE06D8047002264305141DC
S214014B40A064E1648BE05120205C012804D005209C
S214014B50C0435021605482E0A06B864200D07EE0C4
S214014B60D2B269462000FFF782FE0321C943020044
S214014B700B0052B29A4204D15020215451202554A0
S214014B806DE040B2002826D1E06D804700226430F7
S214014B905141A064E1644420205A4221615A88426E
S214014BA003D302205121605415E06078002812D00A
S214014BB04720205C401E472160544720205C002887
S214014BC009D160784721605401234720225C0021E7
S214014BD02000FFF7D4FC42E03420205C01283ED1BF
S214014BE0D2B269462000FFF790FE40B2002835D1C8
S214014BF0E06D80470022643051412200283203C212
S214014C00083A0F2039780140022906D10720C0430F
S214014C10206302203421605420E0397801400129C4
S214014C200CD1E07F401CE077E07F022816DB0620EF
S214014C30C04320630220342160540FE039780142DA
S214014C400CD17878002802D18048A08301E07878DA
S214014C50A083B878FFF784FCA077E577FFE7F7BD78
S214014C6038AB01006CAB010070B50024250051255E
S214014C70455D022D02D00420C04325E0856B866881
S214014C80B54201D1012500E025000D704221415AAF
S214014C901D000E00ADB2B6B2B54200D21900230017
S214014CA007E0C56B1E00B6B2AD5D1E00B6B29555E7
S214014CB05B1C1D000E00ADB2B6B2B542F1D3049A2C
S214014CC0118051214454002070BD70B402000B00C5
S214014CD018781070587850705868506098689060CE
S214014CE0D868D06018691061988A908200242000E4
S214014CF0D082200010832000907620009083200030
S214014D0090772000D077002000211500203503C5BC
S214014D10083D1500283503C5083D146325003426D3
S214014D2095559D69D5639D8B402695532500422652
S214014D30955325004426955325004626955525006E
S214014D40472695559064D164200050215054512037
S214014D501454186A5065586A9065986AD06570BC94
S214014D60704738B504003420205C012856D1374DF1
S214014D70A08BA84202D0A08B00283DD0A07F00289F
S214014D800ED0A07F002837D0E06D80472200203269
S214014D900CCA121A8B41002B2EDC01DB002A2BD207
S214014DA02000FFF78AFC40B2002822D1A08BA8423F
S214014DB002D0A08B4019A083E06D804700226430AA
S214014DC051412200283203C2083AE06D80470200B2
S214014DD00B00A07F0021801859412200203203C217
S214014DE0083A208BE18A884206D300203421605499
S214014DF002E0022034216054E06D80472200283210
S214014E000CCA121A8B41002B08DC01DB002A05D2E2
S214014E100120C04320630220342160545120205CCD
S214014E20012811D1E06D8047A26CE36C121A8B4108
S214014E30002B09DC01DB002A06D20220C0435021E8
S214014E40605400205121605431BD0000FFFF000076
S214014E5000B5BFF34F8F054805490860BFF34F8F74
S214014E6000BFFDE701604260836070470400FA05F9
S214014E700CED00E038B504002F48A2688023D0501E
S214014E80C9B200295AD0022900D17FE06AD3042989
S214014E9000D1A3E000D28DE0062900D1C6E000D201
S214014EA0B0E0082900D1E9E000D2D3E00A2900D118
S214014EB00CE100D2F6E00C2900D12FE100D219E175
S214014EC00E2900D152E100D23CE1102900D175E152
S214014ED000D25FE1122900D198E100D282E11429C3
S214014EE000D1BBE100D2A5E1162900D1DEE100D256
S214014EF0C8E1182900D101E200D2EBE11A2900D15C
S214014F0024E200D20EE21C2900D147E200D231E2AF
S214014F101E2900D172E200D258E2202900D19DE27A
S214014F2000D283E2222900D1C8E200D2AEE22329D0
S214014F3000D1DBE2DDE200BF5245535501200100FE
S214014F40A26853680125AB43C9B2014019435160B9
S214014F500021A26853680125AB43C9B20840184333
S214014F605060C6E201200100A26893680125AB43A8
S214014F70C9B20140194391600021A26893680125D6
S214014F80AB43C9B2084018439060B2E20120010069
S214014F90A268D3680125AB43C9B201401943D16069
S214014FA00021A268D3680125AB43C9B20840184363
S214014FB0D0609EE201200100A26813690125AB437F
S214014FC0C9B20140194311610021A2681369012584
S214014FD0AB43C9B20840184310618AE201200100C0
S214014FE0A26853690125AB43C9B201401943516117
S214014FF00021A26853690125AB43C9B20840184392
S214015000506176E201200100A26893690125AB4355
S214015010C9B20140194391610021A2689369012533
S214015020AB43C9B208401843906162E20120010017
S214015030A268D3690125AB43C9B201401943D161C6
S2140150400021A268D3690125AB43C9B208401843C1
S214015050D0614EE201200100A268136A0125AB432C
S214015060C9B20140194311620021A268136A0125E1
S214015070AB43C9B20840184310623AE2012001006E
S214015080A268D36A0125AB43C9B201401943D16274
S2140150900021A268D36A0125AB43C9B20840184370
S2140150A0D06226E201200100626813680125AB4345
S2140150B0C9B20140194311600021626813680125D5
S2140150C0AB43C9B208401843106012E20120010048
S2140150D0626853680125AB43C9B201401943516068
S2140150E00021626853680125AB43C9B208401843E2
S2140150F05060FEE101200100626813690125AB439F
S214015100C9B2014019431161002162681369012582
S214015110AB43C9B2084018431061EAE1012001001F
S214015120626853690125AB43C9B201401943516115
S2140151300021626853690125AB43C9B20840184390
S2140151405061D6E101200100626893690125AB43F5
S214015150C9B2014019439161002162689369012532
S214015160AB43C9B2084018439061C2E10120010077
S2140151706268D3690125AB43C9B201401943D161C5
S21401518000216268D3690125AB43C9B208401843C0
S214015190D061AEE1012001006268136A0125AB43CC
S2140151A0C9B201401943116200216268136A0125E0
S2140151B0AB43C9B20840184310629AE101200100CE
S2140151C06268936A0125AB43C9B2014019439162F3
S2140151D000216268936A0125AB43C9B208401843AF
S2140151E0906286E1012001006268136B0125AB43E2
S2140151F0C9B201401943116300216268136B01258E
S214015200AB43C9B208401843106372E101200100A4
S2140152106268536B0125AB43C9B201401943516320
S21401522000216268536B0125AB43C9B2084018439D
S21401523050635EE1012001006268136C0125AB43F7
S214015240C9B201401943116400216268136C01253B
S214015250AB43C9B20840184310644AE1012001007B
S2140152606268536C0125AB43C9B2014019435164CE
S21401527000216268536C0125AB43C9B2084018434C
S214015280506436E1012001006268936C0125AB434E
S214015290C9B201401943916400216268936C0125EB
S2140152A0AB43C9B208401843906422E101200100D3
S2140152B06268136D0125AB43C9B2014019431165FC
S2140152C000216268136D0125AB43C9B2084018433B
S2140152D010650EE1012001006268136E0125AB43E3
S2140152E0C9B201401943116600216268136E012597
S2140152F0AB43C9B2084018431066FAE0012001002A
S2140153006268536E0125AB43C9B201401943516629
S21401531000216268536E0125AB43C9B208401843A9
S2140153205066E6E0012001006268936E0125AB43FA
S214015330C9B201401943916600216268936E012546
S214015340AB43C9B2084018439066D2E00120010081
S2140153506268D36E0125AB43C9B201401943D166D9
S21401536000216268D36E0125AB43C9B208401843D9
S214015370D066BEE0012001006268136F0125AB43D1
S214015380C9B201401943116700216268136F0125F4
S214015390AB43C9B2084018431067AAE001200100D8
S2140153A062688023D3580125AB43C9B20140194333
S2140153B08023D150002162688023D3580125AB4356
S2140153C0C9B2084018438021505092E001200100E4
S2140153D062688423D3580125AB43C9B201401943FF
S2140153E08423D150002162688423D3580125AB431E
S2140153F0C9B208401843842150507AE001200100C8
S21401540062689023D3580125AB43C9B201401943C2
S2140154109023D150002162689023D3580125AB43D5
S214015420C9B2084018439021505062E001200100A3
S21401543062689C23D3580125AB43C9B20140194386
S2140154409C23D150002162689C23D3580125AB438D
S214015450C9B2084018439C2150504AE0012001007F
S21401546062689423D3580125AB43C9B2014019435E
S2140154709423D150002162689423D3580125AB436D
S214015480C9B2084018439421505032E0012001006F
S2140154906268C823D3580125AB43C9B201401943FA
S2140154A0C823D15000216268C823D3580125AB43D5
S2140154B0C9B208401843C82150501AE00120010023
S2140154C06268CC23D3580125AB43C9B201401943C6
S2140154D0CC23D15000216268CC23D3580125AB439D
S2140154E0C9B208401843CC21505002E0FFF7B0FC87
S2140154F0FFE70020A1688022885031BD016042602C
S214015500704770B50A79002A0DD0022A51D018D3F7
S214015510042A00D1BDE000D283E0062A00D128E1AA
S21401552000D2EEE05DE10021006802691202120A73
S21401553020239A43C9B2490120231940114301612E
S2140155404FE10123026814692402240A2025AC4392
S214015550DBB25B0120252B4023431361002215009B
S21401556003681C692402240A1026B443EDB22D01F7
S2140155701026354025431D61150003681C69240269
S214015580240A0826B443EDB2ED000826354025432B
S2140155901D61098803689C68240C240489B20C43A5
S2140155A09C600068C168090C090492B21143C1608D
S2140155B017E10122150003681C692402240A20262B
S2140155C0B443EDB26D012026354025431D610368C5
S2140155D01C692402240A1025AC43D2B212011025FC
S2140155E02A4022431A610022150003681C6924021E
S2140155F0240A0826B443EDB2ED00082635402543BB
S2140156001D61098803689C68240C240489B20C4334
S2140156109C600068C168090C090492B21143C1601C
S214015620DFE00122150003681C692402240A2026F3
S214015630B443EDB26D012026354025431D6100259A
S21401564003681C692402240A1026B443EDB22D0116
S2140156501026354025431D6103681C692402240A6F
S2140156600825AC43D2B2D20008252A4022431A614B
S2140156700A8803689C68240C240492B214439C6034
S21401568049880068C268120C120489B20A43C260D3
S214015690A7E00122150003681C692402240A2026BB
S2140156A0B443EDB26D012026354025431D6100252A
S2140156B003681C692402240A1026B443EDB22D01A6
S2140156C01026354025431D6103681C692402240AFF
S2140156D00825AC43D2B2D20008252A4022431A61DB
S2140156E04A8803689C68240C240492B214439C6084
S2140156F009880068C268120C120489B20A43C260A3
S2140157006FE00122150003681C692402240A202682
S214015710B443EDB26D012026354025431D611500C9
S21401572003681C692402240A1026B443EDB22D0135
S2140157301026354025431D6103681C692402240A8E
S2140157400825AC43D2B2D20008252A4022431A616A
S2140157500A8803689C68240C240492B214439C6053
S21401576049880068C268120C120489B20A43C260F2
S21401577037E00122150003681C692402240A20264A
S214015780B443EDB26D012026354025431D61150059
S21401579003681C692402240A1026B443EDB22D01C5
S2140157A01026354025431D6103681C692402240A1E
S2140157B00825AC43D2B2D20008252A4022431A61FA
S2140157C04A8803689C68240C240492B214439C60A3
S2140157D009880068C268120C120489B20A43C260C2
S2140157E0FFE770BDF8B504000D0001200300216835
S2140157F04E698E4A3240DBB21B0480267602334065
S21401580013434B612B7821680E68894A3240032680
S214015810B243DBB29B079B0F13430B606978226888
S2140158205368FF26B343C9B219435160A978226869
S2140158305368804E1E40C9B2090231435160EB786D
S21401584021684E687C4A3240DBB21E04FC239B036F
S214015850334013434B602A7921680B691B021B0AEC
S2140158600427FF433B400426D2B2920032401A433B
S2140158700A610100226810690002000A4023984369
S214015880C9B2890140231940014311612F202A5CC6
S2140158906168886920239843D2B2520120231A40B6
S2140158A002438A6130202A5C606881691C2399431F
S2140158B0D2B293001C221A400A43826131202A5C2C
S2140158C06068816903239943D2B29207920F0A4313
S2140158D082612A7B2168486908239843D2B2D200A4
S2140158E008231A4002434A61A91D2000FFF709FE5A
S2140158F0A97B206842691740C9B289000E403E4321
S2140159004661A87B002809D0687B21684A69032381
S2140159109A43C0B28007800F10434861002135E0EA
S2140159200800C0B240002818C37B0A002068160091
S214015930F6B2B600861980277F00F6590F27BE43B8
S214015940DBB21B071B0F3343D2B2920080188022B2
S214015950520083500800C0B240002818067C0A0096
S21401596023681000C0B28000181880277F00C05935
S2140159704027B843F6B2B60140273E400643D2B2AE
S21401598090001818802252008650491C0800C0B2A8
S2140159901028C5DB002021684A69244B1340C0B299
S2140159A0000480225202104018434861F1BD10B530
S2140159B000210A0001221300037004231C00447016
S2140159C0302484700B24C4700C000471C1800181E2
S2140159D00C0084720C0004730C00447382730A007A
S2140159E02F240255302283540A003123C2540A0060
S2140159F00BE01300DBB25B00C318DA730B00140074
S214015A00E4B2640004192374521C1300DBB2102B99
S214015A10EFDB10BD0068C9B289004018C0214900FB
S214015A2040588004800C80B270470000FFFFFEFFE4
S214015A30FFFEFFFFFF00FFFFFFFFC0FFF0B5020004
S214015A4052B2002A16D41822B94B040064B2A40834
S214015A50A4001C59FF25C6001640B540AC43890179
S214015A60C9B2C5002A409140214340B28008800057
S214015A7019501BE00F25AF4B1824020052B22A40E2
S214015A80083A92089200060076B23540083DAD0805
S214015A90AD005D59FF26C7002740BE40B5438901CA
S214015AA0C9B2C0000440A14029439950F0BD80B559
S214015AB0411E80225204914201D301200EE0401E75
S214015AC09D49086003210020C043FFF7B7FF00206F
S214015AD0C34908600720C3490860002002BD10B50D
S214015AE0C14C200000F03AFAC020400024182000E3
S214015AF000F075FC00F00CF800F06CFD00F01EF9EB
S214015B0000F055F8200000F08EFC00F0EAF910BD18
S214015B10F0B585B001246E462000307002277770FC
S214015B202000B080B14D6A4607212800FDF752F8E3
S214015B30200030702000B0806A4613212800FDF74F
S214015B4049F86A4614212800FDF744F86A461521EB
S214015B502800FDF73FF86A4616212800FDF73AF8B7
S214015B606A4617212800FDF735F820003070777057
S214015B700420B0806A4627212800FDF72BF83470F0
S214015B806A4628212800FDF725F8994C22000921AC
S214015B902800FDF706F82068FA218900FDF771F85C
S214015BA0FFF785FF934800F07FFE05B0F0BD38B5DE
S214015BB08D4C2500E03501220021280000F07DFEF5
S214015BC000220021280000F0B7FE01220121280052
S214015BD000F073FE00220121280000F0ADFE012234
S214015BE00221280000F069FE00220221280000F0B0
S214015BF0A3FE01220321280000F05FFE00220321FC
S214015C00280000F099FE01220521280000F055FE2B
S214015C1000220521280000F08FFED8340122012140
S214015C20200000F04AFE00220121200000F084FE40
S214015C3001221021200000F040FE00221021200049
S214015C4000F07AFE01220F21200000F036FE00222D
S214015C500F21200000F070FE31BD80B5C0B20028D3
S214015C600BD002281FD013D3042832D026D30628FF
S214015C7045D039D307284DD057E00221A74800F078
S214015C8075FE002801D1012000E00020C0B24DE0E1
S214015C900321A24800F06AFE002801D1012000E09D
S214015CA00020C0B242E001219C4800F05FFE0028BF
S214015CB001D1012000E00020C0B237E00021974862
S214015CC000F054FE002801D1012000E00020C0B2FF
S214015CD02CE00521914800F049FE002801D1012061
S214015CE000E00020C0B221E001218D4800F03EFE18
S214015CF0002801D1012000E00020C0B216E00F21EB
S214015D00874800F033FE002801D1012000E0002082
S214015D10C0B20BE01021824800F028FE002801D115
S214015D20012000E00020C0B200E0002002BD00001B
S214015D3000E400E01CED00E014E000E0F8B5A2B0DD
S214015D40784800886946088177480390774801902B
S214015D5002A9019800F0A8FF15A8FFF728FE012563
S214015D6015A80570857303242100417300263100B0
S214015D7001730A21C1730B21417415A91A48FFF753
S214015D8031FD6A4628211948FCF70BFF04A801F0EB
S214015D90E1F804AF3000387030003871FD7107202B
S214015DA0F8702000B87102202C2178542D203C5424
S214015DB00098C0092821FCF764FFC821FCF761FFA1
S214015DC03881BE815A4C04A9200001F01BF920003D
S214015DD001F028F86421019801F004F823B0F0BD21
S214015DE018E000E010E000E0C0300020C8300020DD
S214015DF040500020FFFF000038B54E4C4E4D0021AC
S214015E002800FFF707FE206001212800FFF702FEA9
S214015E10606000F059F849490A78002A03D0022A3E
S214015E203DD027D34FE0020092B2454B9A420CDB9D
S214015E3044480288521C02800288434B9A4218DB6F
S214015E40002202800120087013E080B23F4A90428F
S214015E500CDA3C480288521C028002883A4B9A426D
S214015E6007DB002202800220087002E0002035498C
S214015E70088028E080B2FA22920190420BDA31487B
S214015E800288521C028002882F4B9A4206DB0022AF
S214015E9002800A7002E000202A49088013E080B2DE
S214015EA02B4A90420BDB27480288521C028002884C
S214015EB0254B9A4206DB002202800A7002E000208F
S214015EC020490880FFE731BD1A4800682149484348
S214015ED0000BAF218900401880B270471748007840
S214015EE0704700B585B0684600F061FA0120694642
S214015EF002000A7000224A70CA7003000B714A71D0
S214015F0088714A72C82080010490FA2080000390AC
S214015F106946114800F086F905B000BDA0310020A1
S214015F2098310020322D0100B8AC01002C3200203F
S214015F308431002044500020C0300020A6550020A7
S214015F4075400000A2550020210300003421000006
S214015F5029230000D8D6000040320020F0B58BB0CF
S214015F6004007D4D2A007D492000FFF7C7FA7C48D2
S214015F700590069000200790089009900A90794EA7
S214015F80794F05A8039002977848019078480090C9
S214015F903300784A784920000830FCF7DEFD77495F
S214015FA02000383001F03AF9754920003C3001F004
S214015FB037F974492000403001F032F97249200067
S214015FC0443001F02FF9714A71492000483001F040
S214015FD02BF970492000543001F02AF96E4920004F
S214015FE0583001F027F96D4920005C3001F024F9A2
S214015FF032006B492000603001F020F9022069462A
S214016000087404A80390029501970096594B574AC5
S214016010644920008030FCF7E5FF634920009C308E
S21401602001F004FA2A0061492000A03001F00CFAC0
S2140160302A005F492000A83001F009FA5D492000D6
S214016040B03001F007FA5C492000B43001F004FAE0
S2140160505A492000B83001F001FA59492000BC30F5
S21401606001F0FCF957492000C03001F0F9F9564912
S2140160702000C43000F0D4FE544A55492000C830F0
S21401608000F018FC534A54492000D03000F012FCAE
S214016090524A53492000D83000F00CFC514A52496C
S2140160A02000E03000F006FC504A51492000E8305C
S2140160B000F000FC00962E4B3A004E492000F030CE
S2140160C001F0D0F92A004C4980204000201801F048
S2140160D00FFA2A00494984204000201801F008FAE6
S2140160E0244B224A2449882040002018FEF7BAFE95
S2140160F043498E204000201801F026FA4149B2207B
S2140161004000201801F02AFA3F49B4204000201828
S21401611001F024FA2A003D49B6204000201800F07C
S214016120C0FD3B49BA204000201801F031FA394938
S214016130BC204000201801F02BFA3749BE20400051
S214016140201801F025FA3549C0204000201800F03B
S21401615067F80BB0F0BD00BF00F0054000400240FC
S21401616000127A0000E0064000E8064000F806400B
S21401617000E4064000F0064000F0074000400740FB
S214016180003000400040004000C0004000100240C7
S2140161900080004000900140008001400050004017
S2140161A000000240008003400060064000200740D7
S2140161B000300740007007400050074000000340D1
S2140161C00010034000D00040006002400050034031
S2140161D00000064040500340001006408050034037
S2140161E000200640C05003400030064000510340E6
S2140161F00040064000D00740008005400090054062
S2140162000080074000C0024000D0024000E0054088
S21401621000A0064000B0064000C0064000A00740AF
S214016220016070477FB50400206801260068C20936
S2140162303000104022681268530932001A40236861
S2140162401B685D0A33002B40C0B2002800D0ADE0C9
S214016250D2B2012A00D0A9E0DBB2012B00D0A5E022
S2140162600D0010220021684601F0B6F90098704929
S214016270014000912A78684603686E491940D2B2F7
S2140162801304E022D2021A400A4302606A78684682
S214016290036869491940D2B2D20380231B021A400F
S2140162A00A430260EA786846036864491940D2B234
S2140162B0120380235B011A400A4302606A7968462A
S2140162C0016840239943D2B2920140231A400A43FF
S2140162D00260AA796846016820239943D2B2520126
S2140162E020231A400A4302602A7A6846016802237C
S2140162F09943D2B2520002231A400A430260687AD6
S21401630069460A6801239A43C0B2304010430860C8
S214016310AA78684603684A49194092B292038023D4
S214016320DB011A400A4302602A7968460168802325
S2140163309943D2B2D20180231A400A430260EA7915
S2140163406846016818239943D2B2D30018221A402E
S2140163500A4302603B482168486000992268116040
S214016360296922689160216809688A0A310011400A
S214016370C9B20029F7D0216809684A0A31001140DC
S214016380C9B20029F7D0697800290FD02E492268B2
S214016390516021684860E8682168C8602068006824
S2140163A0410A30000840C0B20028F7D07FBD012165
S2140163B00A0002700022130043700B008370130062
S2140163C0C3701300037113004371817111000172D0
S2140163D0110041721D490161C260C271704700B56A
S2140163E002680121126852090A40D2B2012A19D163
S2140163F0144A03685A600268126880239A43036845
S2140164001A60124A03689A6002681268D20A0A4041
S214016410D2B2002AF8D102681268520A0A40D2B2F1
S214016420002AF8D000BD08490068416070470000A6
S214016430846FF8FFFFFFF8FFFF7FFFFFFFEFFFFF0F
S214016440FFBFFFFF20C528D902A680B4FFFF0000CA
S214016450F8B594B000200020694608704CE001A908
S2140164602868FDF772FB42E001AE6846007830709E
S214016470964D01A92868FDF7ABFB002837D0D02040
S214016480205869460978142251434018407A012859
S214016490E5D101A92868FDF758FB01A92868FDF791
S2140164A0F4FA4820325C01A801000831884C982093
S2140164B04001251828784C2358432018071D38001A
S2140164C001F0AEF8029829784C22514360502878A2
S2140164D04C214843201844214822B25C4254287873
S2140164E0401C28702878202801D300202870684690
S2140164F00078401C69460870764C68460078CC21C6
S214016500615C8842B0D315B0F0BD70B501000024BF
S21401651020006F4BC14A9D18982252019A5C2E7832
S214016520B24211D04C2228784C26704318180E001F
S2140165300100300001F074F82878401C2870287893
S214016540202800D32C700120C0B270BDF0B593B0E6
S21401655000242300DBB22500EDB2E4B200E0641CA7
S2140165605C4D2600CC27EF5DF6B2BE420CD2D0269B
S214016570AE59B4462700FFB2142677436646F6198D
S2140165807668B042EBD123002800D0306C4605680F
S2140165901E00F6B214277E43AD5B25704825625572
S2140165A00068DBB214246343C01840680190D2B27D
S2140165B0684604000834200001F032F8434C69466E
S2140165C02068FDF712FA69462068FDF703FA0020F5
S2140165D013B0F0BDFEB50025029591492A003C4C4A
S2140165E0200001F02BF8D8212A003A4C2600300072
S2140165F001F024F88B4E30008030344908608A4F11
S21401660001220921380000F058F901220921380039
S21401661000F092F900220921380000F09AF9834F20
S21401662005220021380000F048F905220121380032
S21401663000F043F92000FCF7E4FC0820CC2160546C
S2140166407B48D02160500120010021702900617033
S2140166502900A1702900E17030216554C8216054D9
S21401666002AA0B2130000830FCF79BFA607801285B
S2140166700BD101200190FA20C00000906D4B6E4AAC
S214016680029920001C30FDF7C6FB002001906B48E4
S2140166900090684B6A4A029920000830FDF7BBFB60
S2140166A021000A480068FCF7C1FD092000F0FCF84B
S2140166B0F7BD10B50400FFF711FC002804D108222D
S2140166C021006048FFF742FF10BD00003450002053
S2140166D0583C00205C4F00207CB5050008242100B2
S2140166E000226E46300000F0A9FF022001F008F8F3
S2140166F069460978084369460870032001F000F8E6
S214016700694609784000084369460870002000F091
S214016710F7FF69460978800008436946087001203A
S21401672000F0EEFF69460978C00008436946087024
S214016730042000F0E5FF6946097800010843694630
S2140167400870052000F0DCFF69460978400108431F
S21401675069460870062000F0D3FF69460978800173
S214016760084369460870072000F0CAFF69460978A1
S214016770C00108436946087022006946280000F0F7
S2140167804FFF73BD30B593B02F4C2000FFF7A4FF29
S21401679020788006800E00280DD02C4D2888642194
S2140167A0FCF76CFA002902D12000FFF782FF288847
S2140167B0401C288002E0002024490880062000F0C2
S2140167C08FFF002804D1072000F08AFF002802D09E
S2140167D02000FFF76EFF1D480188FA2292009142C1
S2140167E001DB002101806846FFF78FFE01280FD1EB
S2140167F000981749884203D000981649884207D165
S21401680068464421435C021D00991348FEF706F9C9
S214016810124801F07AF813B030BD000001130000F1
S21401682004130000C0300020983100209031002071
S21401683050A801004C1D000080841E00C409000001
S21401684020A107000102000038500020A0550020BA
S21401685031070000DF07000020200020082000206C
S21401686000B5010049B2002905D40121C006C00EB9
S21401687081400B48016000BD00B50A480168012946
S21401688006DB0168491E01600068012800DA62B66D
S21401689000BD000072B603480168491C01607047DC
S2140168A000E100E06450002080B540B2FFF7D8FF59
S2140168B001BD7047016042607047F0B51300DBB25E
S2140168C0002B1BD10B0004689D006659194D3540FD
S2140168D0D2B21602E022D20032402A439B00E25096
S2140168E0012200688B00C3580424A343D2B292004D
S2140168F0042422401A43890042501AE000260C0064
S2140169000568A300EB580427BB43F6B2B60004277C
S2140169103E401E43A300EE5000688B00C358054C52
S2140169201C40D2B21302E022D2001A402243890050
S2140169304250F0BDFFF8FFFF10B443685B690124C5
S2140169408C40A343D2B28A401A434068426110BCCD
S214016950704710B443681B6801248C40A343D2B22D
S2140169608A401A434068026010BC704710B50200A6
S2140169700020030052681469012213008B40234053
S214016980002B00D01000C0B210BD00000068C00F80
S214016990C0B27047026852005208C9B2C907114313
S2140169A0016070470268A14B1340C9B20A06FE2176
S2140169B0C90511401943016070470268A24B134094
S2140169C0C9B20A04FE21C903114019430160704788
S2140169D002689E4B1340C9B20A02FE21C90111404A
S2140169E019430160704702687F239A43C9B249067A
S2140169F0490E1143016070474068C00FC0B270472E
S214016A00426852005208C9B2C90711434160704733
S214016A104268864B1340C9B20A06FE21C9051140D9
S214016A201943416070474268874B1340C9B20A0454
S214016A30FE21C90311401943416070474268834BE8
S214016A401340C9B20A02FE21C9011140194341602F
S214016A50704742687F239A43C9B24906490E1143DB
S214016A6041607047C068C00FC0B27047C26852002C
S214016A705208C9B2C9071143C1607047C2686B4B5F
S214016A801340C9B20A06FE21C90511401943C16067
S214016A907047C2686C4B1340C9B20A04FE21C90391
S214016AA011401943C1607047C268684B1340C9B2B0
S214016AB00A02FE21C90111401943C1607047C2682C
S214016AC07F239A43C9B24906490E1143C1607047F4
S214016AD04069C00FC0B27047426952005208C9B23D
S214016AE0C90711434161704742697F239A43C9B27E
S214016AF04906490E1143416170478069C00FC0B213
S214016B007047826952005208C9B2C90711438161B0
S214016B1070478269454B1340C9B20A06FE21C90572
S214016B2011401943816170478269474B1340C9B2CE
S214016B300A04FE21C9031140194381617047826925
S214016B40424B1340C9B20A02FE21C9011140194342
S214016B508161704782697F239A43C9B24906490E0B
S214016B60114381617047C069C00FC0B27047C269E6
S214016B7052005208C9B2C9071143C1617047C269C0
S214016B802A4B1340C9B20A06FE21C9051140194312
S214016B90C1617047C2692C4B1340C9B20A04FE2179
S214016BA0C90311401943C1617047C269274B13409D
S214016BB0C9B20A02FE21C90111401943C1617047D9
S214016BC0C2697F239A43C9B24906490E1143C1617E
S214016BD07047806AC00FC0B27047826A520052087E
S214016BE0C9B2C907114381627047826A7F239A43FB
S214016BF0C9B24906490E114381627047006BC00F46
S214016C00C0B27047026B52005208C9B2C90711439D
S214016C1001637047026B054B1340C9B20A06FE2199
S214016C20C90511401943016370470000FFFFFF804B
S214016C30026B054B1340C9B20A04FE21C903114079
S214016C401943016370470000FFFF80FFFF80FFFFCD
S214016C50026B604B1340C9B20A02FE21C901114002
S214016C60194301637047026B7F239A43C9B24906F1
S214016C70490E114301637047406BC00FC0B27047A5
S214016C80426B52005208C9B2C907114341637047AB
S214016C90426B7F239A43C9B24906490E11434163A9
S214016CA07047016042607047F8B50600002E05D0B7
S214016CB00D00002D02D02888002800D133E00027DF
S214016CC03C0010E06868210089B203224A4380181C
S214016CD042786868210089B203234B43C15C3000C7
S214016CE000F022F8641C2000298880B28842E9D38B
S214016CF03C0013E06868210089B203224A438018E9
S214016D008078002809D06868210089B203224A43A6
S214016D1080184178300000F033F8641C2000298880
S214016D2080B28842E6D3F1BD70B506000C001500AE
S214016D302900C9B2300000F034F8012801D1002042
S214016D401CE02800C0B28208AB079B0F224D100042
S214016D50C0B2000128181900C9B28900405800289D
S214016D600BD02100C9B23068D2B21201AA18DBB228
S214016D709B00D2589047012000E00020C0B270BDB1
S214016D8080B5C9B28B08154A1900C9B28900515895
S214016D90002905D001210068DBB29B00D25890473C
S214016DA001BD38B5020001242000C9B289080C4B88
S214016DB00D00EDB2AD005D59002D09D01068C9B2C5
S214016DC0890059588847012801D1200000E0002099
S214016DD0C0B232BDFF80FFFFB4A6010000AB0100C8
S214016DE0C8AA010078B500231C0045686E6C012214
S214016DF096430122E4B2144034436C64009302E0EB
S214016E00009B5B1C0093009B8B42F9D311004068EA
S214016E10436C0124A343C9B20A401A43426471BDBC
S214016E200160704701210068026880239A43C9B255
S214016E30C901802319401143016070470021006891
S214016E40026880239A43C9B2C901802319401143BD
S214016E5001607047006801680122914301220A43DC
S214016E6002607047F3B581B000210A003AE06D4632
S214016E702A70019D2D686E46367828277E43AE1906
S214016E8037695E4E3E40C0B2000430436E463678E7
S214016E9028277E43AD1928611000019D2D68060044
S214016EA0F6B228277E43AE193769554E3E40E4B206
S214016EB024023443C0B22826704328180461100007
S214016EC0019C24680500EDB22826754365192D69D5
S214016ED0FF26B543DBB22B43C0B2282568432018F2
S214016EE00361521C1000C0B2022831DA0C000B00FC
S214016EF008000D0009E007E001261F003300AB4043
S214016F003B43AE40064330006D1C2E00F6B2082E01
S214016F10ADDA029E1700FFB2FF00F6192F00FFB28E
S214016F20F65D002E05D0022E09D003D3032EE3D042
S214016F30E1E7E9E71E000123AB403343E4E701261E
S214016F401F003300AB403B43AE4026433400DBE733
S214016F50F7BD0000F0B500210A0002700A00427079
S214016F600A0082700A00C2700F2202710A00427182
S214016F700A00827101221300C371A24B0381418171
S214016F800B0018E01D00EDB2ED0045192600F6B223
S214016F90AD192C260F00AF551D00EDB22D01451978
S214016FA02600F6B27600AD19A981641C2500EDB263
S214016FB0082DE7DB5B1C1C00E4B2022C01DA0C0096
S214016FC0F4E72C23C2540A0011E00B001400E4B2CB
S214016FD004193C2563551300DBB25B00C318D9873F
S214016FE01300DBB25B00C31840241953521C130074
S214016FF0DBB2002BE9D0F0BD00000000FFFF00FF70
S214017000FF00FFFFF3B581B004002000FFF716FF75
S2140170100298008921684A68120C120480B2024361
S2140170204A60029840892168CA68120C120480B22C
S2140170300243CA6000212AE01300684601700298E4
S2140170400D00EDB22D0140191500EDB26D0040198D
S21401705086892568684600782827784328181F00FF
S214017060FFB2BF00C0198069000C0004B6B23043FD
S2140170706E46367828277E43AD19DBB29B00EB18A7
S2140170809861521C1000C0B20828D5DB491C0800C4
S214017090C0B2022801DA0022F4E7029801002C317E
S2140170A02000FFF7DFFE0298407821680A68564BF9
S2140170B01340C0B240048022920210401843086078
S2140170C00298807821680A68504B1340C0B2C0030A
S2140170D0802212021040184308600298C078216886
S2140170E00A684B4B1340C0B20203E020C0011040B7
S2140170F0184308600298007921680A68454B1340D6
S214017100C0B20202F0200001104018430860029845
S214017110407921680A6820239A43C0B2400120239F
S2140171201840104308600298807921680A680C2389
S2140171309A43C0B283000C2018401043086002989E
S214017140C07921680A6802239A43C0B2400002232C
S21401715018401043086000252800290023E0029A01
S2140171600B00DBB25B00D218D28F1204029B0E001A
S214017170F6B276009B1940269B5B1A430B002668E5
S214017180DBB29B00F318CA2676009A51029A0B00CE
S214017190DBB2D2183C23D25C002A03D002000120C5
S2140171A088401043491C0A00D2B2002AD7D0216871
S2140171B0C82252008A58FF239A43C0B21043C822FD
S2140171C0520088502000FFF72DFE280021680A682B
S2140171D0114D2A40C0263603C0B280043040104309
S2140171E008602000FFF736FE2000FFF727FE029812
S2140171F0007821680A681540C0B2800406402E4314
S2140172000E60F7BD60EA0000FFFFFDFFFF7FFFFF96
S214017210FF8FFFFFFFF0FFFFFFFFF3FF01607047E7
S21401722001607047016070474160826070470000EE
S21401723001607047016070470160704738B504000F
S214017240216062600025A560E0208002E060802069
S21401725040052061802000026061200000F0C8F82F
S2140172602076E561207E002800D06561200000F0D0
S21401727001F831BD30B401221300046800210D006D
S214017280DBB25B0002252B402360130004680D006F
S214017290DBB21B0110252B402360130004680D0090
S2140172A0DBB25B0120252B402360130004680D0030
S2140172B0DBB29B0140252B402360130004680D00C0
S2140172C0DBB2DB0008252B4023600068D2B29100B8
S2140172D004221140016030BC704730B50100002324
S2140172E01800012214000D68E4B2E3018024234053
S2140172F02B600B681B68DB091340DBB2002BF8D050
S2140173000B681B685B091340DBB2002B0CD10B68C2
S2140173101B681B091340DBB2002B05D109680968FD
S2140173201140C9B2002900D01000C0B230BDF6B578
S21401733083B001000024200022006A46127C402A05
S21401734000DB01200293029A002A00D1012000915D
S2140173500100C9B2002935D10098006801250068EE
S214017360C10928000840C0B2002801D1022029E046
S2140173700098FFF77FFF082321000098026820008D
S214017380FF2001900E00F6B29619367F019FBE438C
S214017390DBB2019F1F403743C9B251180F776946C8
S2140173A0097C009A126823002B00DBB2D3181B7FDE
S2140173B08343C9B208401843EDB2511908770098C3
S2140173C0FFF78BFF0100C9B200290ED121000AE0A8
S2140173D00A00D21D009B1B682500D2B29A18127FA4
S2140173E0029B5A54491C0829F2D3C0B205B0F0BD1D
S2140173F03EB5050008220021684600F0EDF80020A1
S2140174000400FF20694608706B4600220021280010
S214017410FFF78DFFC0B2002804D1684600788007C8
S21401742000D401242000C0B23EBD0000016000214E
S2140174300168CA6E01239A43CA660068016C0A0095
S214017440D207D20F006C704701604260704701603E
S2140174504260704701607047016070470160704785
S2140174600160704710B4019C016042608360C46093
S21401747010BC704702692F4B1340C9B20A06F021AF
S2140174800905114019430161704702692A4B1340EF
S214017490C9B20A04F021090311401943016170477A
S2140174A00269264B1340C9B20A02F02109011140B4
S2140174B019430161704702690F239A43C9B209074C
S2140174C0090F11430161704742691C4B1340C9B251
S2140174D00A02F021090111401943416170474269CE
S2140174E00F239A43C9B20907090F11434161704737
S2140174F038B5050029606A60002408E010482100BC
S21401750089B2425C0C21280000F006F8641C2000B9
S21401751080B20628F2D331BD80B51300DBB2062B4C
S21401752006DAC9B24068074BD2B292009A58904721
S21401753001BD0000FFFFFFF0FFFFF0FFFFF0FFFFC0
S214017540A8AC010068AC0100016000210171417125
S2140175502822815438228154704700000160016856
S2140175600A6980235B0013430B6101680A69802363
S2140175709B0013430B61012101680A69022313432F
S2140175800B6100BF00BF00BF0021006801617047AA
S21401759001600168CA6A80231B021343CB6200BFE5
S2140175A000BF00BF00BF0A4B1340CB620168CA6A26
S2140175B08023DB011343CB6200BF00BF00BF00BFC7
S2140175C0044B1340CB620021006801607047000045
S2140175D0FF7FFFFFFFBFFFFF10B50400080011008B
S2140175E00200200000F02AF8200010BD70B4103A06
S2140175F003D378C9103A78C0FBD2530701D318C910
S21401760018C001D508C908C0D20704D30B88038067
S214017610891C801C002A01D50B78037070BC70474A
S2140176208B0701D18307E1D0124205D00B78491CA4
S2140176300370401C521EF9D1704700001206130A4F
S2140176401A43130C1A4300BF094205D0830705D01D
S2140176500270401C491EF9D1704700001300103912
S21401766006D330B41400150010393CC0FCD230BC2F
S214017670490700D30CC000D504C0890002D302809C
S214017680801C002900D502707047000000B500205C
S21401769001000CE04C4A0B00DBB2D0544B4A0B0005
S2140176A0DBB2D0544A4A0B00DBB2D054491C0A0064
S2140176B0D2B2082AEEDB00BD00B50100C9B2082926
S2140176C003DA0121414AC0B2115400BD00B50100E0
S2140176D0C9B2082903DA01213D4AC0B2115400BDDE
S2140176E000B50100002210000B00DBB2082B05DA02
S2140176F0364B0800C0B2185CC9B25A54C0B200BDBD
S21401770000B50100C9B2082903DA2F49C0B2085CE6
S21401771000E0002000BD70B50024250022E02A4EBE
S2140177202800C0B2305C012803D12800C0B2FFF7A0
S214017730CDFF20002900C9B2705412E0C0B2002863
S2140177400FD124482900C9B24900415A0029E6D080
S2140177502900C9B24900415A491E2A00D2B2520034
S21401776081526D1C2800C0B208282BDA2800C0B24E
S214017770FEF773FA0100C9B20129DFD112492A00C6
S214017780D2B28A5C012AD9D012482A00D2B252005B
S214017790825A521C2B00DBB25B00C2522A00D2B2C4
S2140177A05200825A142ADCDB01222B00DBB2CA54B7
S2140177B014212A00D2B2520081522800C0B2FFF72B
S2140177C07BFFCEE770BD000068500020705000209F
S2140177D078500020805000200021016041600A009E
S2140177E002724172704700220260416001210172FB
S2140177F042727047407A7047FEB505000E001400CD
S214017800082100226F463800FFF718FF2000C0B29B
S214017810782805D06F48295A6F482818FFF7E3FFE4
S2140178207920285C002814D02000C0B211280FD07F
S2140178302000C0B212280BD02000C0B2312807D0D9
S2140178402000C0B27E2803D02000C0B27F2800D11D
S2140178500AE068467F2101704670847003226946FB
S21401786028001830FDF761F8F7BD10B500221300A7
S21401787000E0521C13009BB24468A3420AD28368FC
S2140178801400A4B2E4001B5D0C00E4B2A342F0D1E4
S214017890012000E0002010BD70B505000C0021009D
S2140178A028001830FDF711FA012068700026300014
S2140178B0A8703000782168540020002184225201EB
S2140178C0AA1803C2083AA08D44496852E08D44497B
S2140178D06852208E3F49685242482818FFF77CFFBD
S2140178E041482818FFF778FF3B482818FFF774FF30
S2140178F03000300004E031002A187B23D154401CAC
S214017900802149018842F6D370BD7CB5040000256C
S21401791028006946888028002800280020001830A2
S214017920FDF71FFA01A8009080235B0122007B323D
S2140179302100793120001830FDF796F940B2002871
S21401794039D17B20265C3100C9B22000FFF78DFFBC
S21401795000282AD02B0000E05B1C606883422AD2F4
S214017960A068D900405C3100C9B28842F4D1A06851
S214017970D90040188078002806D07C20205CC0B250
S214017980C0097821605402E028007821605418006C
S2140179907A2160546846828821007B312000A668DF
S2140179A0DB00F3185B68984705E011223100C9B285
S2140179B02000FFF721FF08482018FFF71BFF0128CA
S2140179C006D101206070A57003482018FFF704FF58
S2140179D073BD00008C100000A81000008810000085
S2140179E08A100000901000009C10000010B50400E2
S2140179F0A26863681000401C834206D32068815445
S214017A00521CA260E068401CE060A0686168884281
S214017A100DD1A2682168206900F0CCFAA1688842DD
S214017A2003D00020C043E06001E00020A06010BD4C
S214017A30F7B582B005001F0003980124012603E074
S214017A400499FBF71EF9761C04998842F8D2BE42C7
S214017A5000D23E0001950A9D0B98C0071BD4002D4D
S214017A6019D00B98800705D5002F03D13020694621
S214017A70087002E0202069460870002D0BD0AE4247
S214017A8009D26D1E684601780198FFF7AFFF01988D
S214017A90C0680028F1D50198C068002839D402E0F2
S214017AA07F1E04984443022FFAD203982100FBF765
S214017AB0E8F804998842F4D203982100FBF7E1F82C
S214017AC00100039A08006043101A03901248415CB3
S214017AD00198FFF78BFF0198C068002807D42000A3
S214017AE00499FBF7CEF80400002CE5D1FFE70B98CC
S214017AF0C0070ED5002D0CD0002D0AD0AE4208D2FC
S214017B006D1E20210198FFF771FF0198C0680028BB
S214017B10F2D505B0F0BD000080AC0100F1B584B02F
S214017B200E001D00002E01D5704200E03000012439
S214017B30039203E00399FBF7A1F8641C03998842BA
S214017B40F8DA02950298844200D2029C0A9D0B9FA5
S214017B50002D04D0002E01D4780700D56D1EB8077D
S214017B6002D50298002810D0F8070ED4002D0CD0AC
S214017B70002D0AD0AC4208D26D1E20210498FFF7D2
S214017B8035FF0498C0680028F2D50498C06800281C
S214017B9034D4002E06D5704206002D210498FFF736
S214017BA025FF05E0780703D52B210498FFF71EFF74
S214017BB00498C068002821D4B807800F022811D184
S214017BC0029800280ED1002D0CD0002D0AD0AC4210
S214017BD008D26D1E30210498FFF708FF0498C0688C
S214017BE00028F2D50498C068002807D401970095AC
S214017BF0029B039A31000498FFF71AFF05B0F0BD07
S214017C00F1B598B00C00160007A80290402003902A
S214017C10002704971898069005972178641C080099
S214017C20C0B2002808D00800C0B2252800D0C7E09E
S214017C3038000122110000E0CAE02378DBB2232BD2
S214017C4013D02B2B0CD02D2B02D0302B03D011E0D0
S214017C501043641C0FE0030002201843641C0AE072
S214017C60030004201843641C05E0030008201843A1
S214017C70641C00E039000029DFD13A0005E0641CED
S214017C800A235A43C9B25218303A21780B00DBB2A4
S214017C90303B0A2BF3D33B002178C9B22E290DD1F4
S214017CA0641C05E0641C0A256B43C9B25B18303BB3
S214017CB021780D00EDB2303D0A2DF3D3217801E095
S214017CC0641C21780D00EDB26C2DF9D00D00EDB2DB
S214017CD0682DF5D0C9B225296BD0582934D063292F
S214017CE00AD0642914D0702952D073293AD0752944
S214017CF01CD0782928D061E030683060306801688F
S214017D003068001D3060C9B202A8FFF76FFE55E06B
S214017D10316831603168096835682D1D356001901C
S214017D2000920A2202A8FFF7F9FE47E031683160A7
S214017D303168096835682D1D3560019000920A2268
S214017D4002A8FFF775FE39E03168316031680968CD
S214017D5035682D1D356001900092102202A8FFF7AC
S214017D6067FE2BE030683060306805683068001DBB
S214017D70306029786D1C0800C0B2002807D0C9B24F
S214017D8002A8FFF733FE05980028F2D5FFE715E0B5
S214017D9030683060306801683068001D306000204F
S214017DA00190082000900823102202A8FFF740FE49
S214017DB004E0252102A8FFF719FEFFE7641C03E093
S214017DC0C9B202A8FFF712FE0598002800D424E7DE
S214017DD0059801280BDB0498002804D0049A07A90B
S214017DE0189800F0E7F8059804994018059005984A
S214017DF019B0F0BD0CB480B502AA00926A46FFF72E
S214017E00FFFE019904B0084710B5494C03202061D4
S214017E1060614848A0614849E1618021C90021624A
S214017E200021A1626162E16220664448606610201A
S214017E30A0662167E166616741A1E01D00F0D8F800
S214017E404049200000F0D4F82020A07110BDF8B5FC
S214017E5084B004000D00160000200190E768206938
S214017E60874202D2C01B401E03E0A168C91B081846
S214017E70401EA168C91B884201D3A068C01BB0423E
S214017E8001D2009000E000966068C0190099039145
S214017E9029000290039A0298FFF7C2FB0298019804
S214017EA000994018019000982D180098361A0098ED
S214017EB03F18A068874200D10027E760002ECED188
S214017EC0019805B0F0BDF8B504000F001500E6688E
S214017ED0A068801B0090009885420AD260688019CD
S214017EE02A00390007003800FFF79AFB7019E06096
S214017EF010E0009A6068861939003000FFF790FBA1
S214017F0000982D1A66682A00009839183000FFF785
S214017F1087FBE560F1BD00B50169C2688A4204D3FA
S214017F208068401E801A401801E0881A401E00BD75
S214017F30905000209CAC010038510020385500209C
S214017F4052545400B0AC0100F8B516000F00254994
S214017F50182250430818050018356869002803D010
S214017F6002281DD00ED322E02800FFF7D4FFB0422E
S214017F7001D2002405E03400320039002800FFF762
S214017F80A2FF15E02800FFF7C6FFB04201D20400A9
S214017F9000E03400220039002800FFF794FF07E0D4
S214017FA0320039002800FFF752FF040000E00024E9
S214017FB02000F2BD70B504000D00160009480078D7
S214017FC0002801D1FFF720FF320029002000EFF33F
S214017FD01084012383F31088FFF7B6FF84F310881B
S214017FE070BD00009050002080B5FFF70DFF01BD69
S214017FF031B48B0707D00B780370002B20D0401CC0
S214018000491C8B07F7D1164CE501830722D104C919
S214018010131B93432B4205D104C004C9131B93437E
S2140180202B42F9D0FF231A42027009D0120A1A42D3
S214018030427005D0120A1A42827001D0120AC2702A
S21401804031BC70470270120A4270120A8270120A1C
S214018050C270001D04C9131B93432B42F2D0E1E703
S2140180600101010100220260416001210172427298
S214018070704770B504000E0015003448215A344884
S2140180802018FFF7EFFF7820205C012806D02A0091
S214018090310092B220001830FCF747FC70BDFEB5E7
S2140180A005000E001400082100226F463800FFF775
S2140180B0C5FA2000C0B2782805D02448295A244899
S2140180C02818FFF7CFFF7920285C002814D020005D
S2140180D0C0B211280FD02000C0B212280BD0200049
S2140180E0C0B2312807D02000C0B27E2803D02000BD
S2140180F0C0B27F2800D10AE068467F210170467031
S21401810084700322694628001830FCF70EFCF7BD80
S2140181107CB56C46AE4D2E682660DBB2042B14D3BC
S214018120069C0B0004210D00258014008078DBB22C
S214018130834204D100222000FFF780FA05E068465A
S2140181400A0001002000FFF76BFA73BD8C100000D7
S214018150A810000001207047F8B584B006000C0096
S2140181601500002008210020009002AF009A380078
S214018170FFF764FA00206946C88000200020280026
S214018180B1687A22B25CD2008918497880B289B285
S214018190884205D2132227213000FFF780FF14E121
S2140181A07078012805D1222227213000FFF777FFBA
S2140181B00BE184204001301803C8FA22D2000023C4
S2140181C0994208DC01DB904205D237222721300094
S2140181D0FFF765FFF9E0200041784906490E6A4637
S2140181E0117167216A4611726946097902AA5170AE
S2140181F069460979C90776D5002738007549087098
S2140182003C0000E0641C2000C0B2042833DA724D42
S214018210684600792100C9B20901695C8842F1D13A
S2140182202000C0B20001281880782100C9B20901D7
S2140182306918497888421ED28420400130180CC83B
S21401824008382000C0B200012818083003C8121AE6
S2140182508B41624800218B4208DC01DB824205D259
S214018260362227213000FFF71AFFAEE02000C0B209
S214018270000128184770E4B2042C05DB31222721BF
S2140182803000FFF70CFFA0E0062301A8801C009039
S214018290DBB202A8821C684601793000FFF738FF7E
S2140182A06846C088002818D06846C288921C92B2D8
S2140182B002A93000FFF7DDFE6846007945490870DF
S2140182C06846C088464908806846C28802A8811C5C
S2140182D0444C2000FFF7A4F977E031222721300033
S2140182E0FFF7DDFE71E03B4C694609792278521CA6
S2140182F0914205D0242227213000FFF7D0FE64E00A
S214018300AD1EADB20095831C3548028835492078EC
S214018310FFF720FFC0B2012821D1022202A93000B6
S214018320FFF7A7FE00200100217069460979491E62
S214018330B17001000A00D2B2042A46DA264A6B4618
S2140183401B790C00E4B22401145DA34205D103009D
S2140183500C00E4B2240112195370491CEAE73522D5
S21401836027213000FFF79BFE00232AE01A4A2078D7
S2140183701900C9B20901515C884221D11800C0B266
S214018380000110184078401C1900C9B209015118A3
S21401839048701800C0B20001101880781900C9B2E0
S2140183A009015118497888420AD2842040013018C0
S2140183B003C81D00EDB22D015219083203C2083A56
S2140183C05B1C1800C0B20428D0DB05B0F0BD00006D
S2140183D0BCAC0100A85500200000002010270000BA
S2140183E0A45500204855002000220260416001216A
S2140183F001724272704770B504000E0015002548E0
S214018400215A25482018FFF7EFFF7820205C012825
S21401841006D02A00310092B220001830FCF785FA07
S21401842070BDFEB505000E001400082100226F463F
S2140184303800FFF703F92000C0B2782805D01548A8
S214018440295A15482818FFF7CFFF7920285C0028FD
S21401845014D02000C0B211280FD02000C0B21228BC
S2140184600BD02000C0B2312807D02000C0B27E2831
S21401847003D02000C0B27F2800D10AE068467F21E1
S2140184800170467084700322694628001830FCF794
S2140184904CFAF7BD8C100000A810000000B50028AB
S2140184A0FFD000BD00B50028FFD000BD00B50028F4
S2140184B0FFD000BD00B50028FFD000BD00B50028E4
S2140184C0FFD000BD00B50028FFD000BD00B50028D4
S2140184D0FFD000BD00B50028FFD000BD00B50028C4
S2140184E0FFD000BDF3B5FFB086B00600140000252E
S2140184F003952800280028002800032069460870F4
S2140185008020800001902A0005AF01993800FFF70E
S21401851095F82800694608812000B1687A22B25C85
S214018520D2008918497880B289B2884205D21322CE
S21401853031213000FFF775FFE5E08698417849065E
S214018540490E6A46517081780902C2788918241F3B
S2140185506A4694806A469288002A01D0001D0390DC
S2140185602C0000E0641C20006A461278C0B29042DB
S21401857029D266482200D2B214235A43825A0B00EB
S2140185809BB29A42EED171782200D2B214235A439A
S21401859082189278914222D12100C9B21422514305
S2140185A04118C97800290ED02100C9B214225143BE
S2140185B04018C078B178884205D033223121300086
S2140185C0FFF72FFF9FE0200069460978C0B2884276
S2140185D00BD3312231213000FFF723FF93E0222213
S2140185E031213000FFF71DFF8DE0802080000490D0
S2140185F02A0005AF04993800FFF720F8684640784E
S214018600012804D066D303284CD027D362E03F4D1F
S21401861002A8009080239B0005AA684681880398DB
S21401862084462700FFB214204743E819876860464E
S214018630B8470120E4B214214C4329190871684651
S214018640008904284CDB6846007D712848D16846BD
S214018650028905A93000FFF7CEFE54E02B48210021
S214018660C9B21422514340180079002819D002A833
S214018670009080239B0005AA684681880398019094
S214018680224884462700FFB2142047436046C0199B
S214018690C7680198B8471D48E4B214214C43001935
S2140186A00571CCE7194D2000C0B2142148432818A3
S2140186B0007900280DD002A8009080239B0005AA0F
S2140186C0684681880398E4B214277C432C192469F0
S2140186D0A047B4E7122231213000FFF7A2FE12E0D4
S2140186E068460089032809D105A801787F2905D1A4
S2140186F0827831213000FFF794FE04E024223121F4
S2140187003000FFF78EFE7FB008B0F0BD8C01002070
S214018710002202604160012101724272704770B509
S21401872004000E001500AE48215AAE482018FFF787
S214018730EFFF7820205C012806D02A00310092B293
S21401874020001830FCF7F1F870BDFEB505000E00EC
S2140187501400082100226F463800FEF76FFF200044
S214018760C0B2782805D09E48295A9E482818FFF797
S214018770CFFF7920285C002814D02000C0B2112831
S2140187800FD02000C0B212280BD02000C0B2312872
S21401879007D02000C0B27E2803D02000C0B27F28B8
S2140187A000D10AE068467F2101704670847003227A
S2140187B0694628001830FCF7B8F8F7BDF6B5FFB0E3
S2140187C082B005000020002000260020002000279F
S2140187D0802189000020009001AC009A2000FEF75D
S2140187E02DFF82A80088A9687A22AA5CD20089187F
S2140187F0497889B2884205D2132222212800FFF740
S214018800A4FFEAE082A80088401EC00705D513220F
S21401881022212800FFF799FFDFE082A800884008A0
S21401882080B2002805D1132222212800FFF78DFFF0
S214018830D3E0622001A9320092B28854761C01204E
S2140188406946088079E0300080B22969220092B238
S21401885014235343C91889894018801C62498842E9
S21401886000DB9FE02869210089B214224A43801860
S2140188708078052800D19BE068782969220092B2A9
S21401888014235343C918C978884200D290E0286956
S214018890210089B214224A4380188289D2B22869FB
S2140188A0210089B214234B43C018816828002F6920
S2140188B0BC462700BFB214237B436746FB181B69DF
S2140188C09847012701A881996A461288895C320077
S2140188D092B28154761C81996A4612888918497821
S2140188E0320092B28154761C68464680286921007F
S2140188F089B214224A43801882892869210089B2E4
S21401890014234B43C018816801A86B465B88C618C0
S2140189103000FEF785FE684640882969A4B2142215
S21401892062438918898946183800C0B2002845D0A4
S21401893068460088801C694608806846008882A9C7
S214018940098888423AD2819869460988405C0002C3
S21401895081996A46128889184978084300242700B5
S21401896000E0641C2100AA8A89B29142DCD22969FE
S214018970220092B214235343C95A020092B2914282
S214018980EFD1A8782969220092B214235343C9185B
S2140189900979884200D156E7332222212800FFF7C1
S2140189A0D4FE1AE0142222212800FFF7CEFE14E09E
S2140189B0222222212800FFF7C8FE0EE0FFB2002F78
S2140189C006D0320092B201A92800FFF7A8FE04E003
S2140189D0312222212800FFF7B8FE7FB004B0F0BD97
S2140189E08C100000A81000000102000000220260A6
S2140189F04160012101724272704770B504000E0099
S214018A0015009548215A95482018FFF7EFFF782062
S214018A10205C012806D02A00310092B220001830CE
S214018A20FBF783FF70BDFEB505000E00140008219C
S214018A3000226F463800FEF701FE2000C0B27828FB
S214018A4005D08548295A85482818FFF7CFFF792091
S214018A50285C002814D02000C0B211280FD02000B6
S214018A60C0B212280BD02000C0B2312807D0200097
S214018A70C0B27E2803D02000C0B27F2800D10AE011
S214018A8068467F210170467084700322694628007B
S214018A901830FBF74AFFF7BD7047704770477047BD
S214018AA0F6B5FFB082B004000D000026300030009D
S214018AB0300002206946087080218900320001AF2B
S214018AC03800FEF7BBFD82A80088A1687A22A25C66
S214018AD0D2008918497889B2884205D213222F21FB
S214018AE02000FFF7A0FFB3E06078012805D122221D
S214018AF02F212000FFF797FFAAE0280041780902FE
S214018B0082788918C2786B465A70350000E06D1C71
S214018B102A006B461B78D2B29A4220D2504A2B00CA
S214018B20DBB214277B43D35A0F00BFB2BB42EED150
S214018B302900C9B2142359435118897800290ED047
S214018B402900C9B21423594351188978A278914251
S214018B5005D033222F212000FFF765FF78E029009A
S214018B606A461278C9B2914205D331222F212000DC
S214018B70FFF759FF6CE001A96F220A7042784A702C
S214018B8082788A70C278CA7069464978002902D00C
S214018B9003291BD057E032482900C9B21422514399
S214018BA04118CE722900C9B21422514341180969ED
S214018BB000290AD0EDB214214D43401900698047BF
S214018BC0042201A92000FFF718FF41E0244E82A9E4
S214018BD009882A00D2B214235A43B218127A121DF7
S214018BE0914205DA22222F212000FFF71CFF2FE0F9
S214018BF001212A00D2B214235A43B218D172290095
S214018C00C9B21422514371180A7A011D2800C0B254
S214018C1014235843301847683800FEF701FD280032
S214018C20C0B2142148433018C06800280AD0EDB2FB
S214018C30142045437019C0688047042201A920000A
S214018C40FFF7DBFE04E031222F212000FFF7EBFEC9
S214018C507FB004B0F0BD00008C100000A81000002A
S214018C606401002001000500000000000000000073
S214018C7000000000030005000000000000000000E6
S214018C8000000000110005000000000000000000C8
S214018C900000000063000500000000000000000066
S214018CA0000000000100000031070000DF0700009F
S214018CB0B1070000503200200002000050340020AE
S214018CC008080000000000004D65010031A3010006
S214018CD03200F401881300001A62040050000000FC
S214018CE0000000001B6304005000000000000000AC
S214018CF01603F00050000000000000001703F0000B
S214018D0050000000000000008873C0005000000002
S214018D10000000000100C10050000000000000003B
S214018D200101C10050000000000000000121C10047
S214018D3050000000000000000127C10050000000A4
S214018D40000000000128C1005000000000000000E3
S214018D500129C10050000000000000000131C100DF
S214018D6050000000000000000041C100500000005B
S214018D70000000000151C10050000000000000008A
S214018D800063C10050000000000000000069C1003F
S214018D9050000000000000000181C10050000000EA
S214018DA0000000000136C200500000000000000074
S214018DB00064C10050000000000000000067C10010
S214018DC0500000000000000092F000005055002006
S214018DD002000000998A01009B8A010020F0000031
S214018DE052550020020000009D8A01009F8A010062
S214018DF000FF0301000000009D840100A58401001E
S214018E00AD84010001FF030100000000B5840100EC
S214018E10BD840100C584010002FF030100000000BB
S214018E20CD840100D5840100DD84010086F10601B0
S214018E300000000060550020010000003BA4010076
S214018E4087F10601000000006155002008000000BF
S214018E5041A4010080F106010000000069550020D0
S214018E600800000031A4010093F106010000000093
S214018E7071550020040000004BA4010095F1060185
S214018E8000000000755500201000000055A40100E8
S214018E9091F1060100000000855500201800000031
S214018EA05FA4010088490870704730B5010089B297
S214018EB0142927DA0021854A0B000400A4B20C25E8
S214018EC065435419237103009BB20C245C431319A8
S214018ED01B1D1C78102525431D7003009BB20C2416
S214018EE05C4313191B1D1C78402525431D70030088
S214018EF09BB20C245C431319D98080B20C234343E4
S214018F00D018017230BD30B50100002210001000EB
S214018F1010000DE06D4B1400A4B20C2565435B19DF
S214018F201B795B065B0EDBB20B4200D0401C521C69
S214018F3013009BB2142BEDDB80B230BDF2B50100FD
S214018F40002318001800180023E01E00B6B20C27F4
S214018F507743EE59360C0700BFB2CE55401C1E00B3
S214018F60B6B20C277743EE59360A0700BFB2CE5584
S214018F70401C1E00B6B20C277743ED590600B6B268
S214018F808D55401C6406640E0500ADB24C55401C60
S214018F905B1C1C00A4B2142C11DA4C4D1C00A4B2AC
S214018FA00C266643AC1924792600F6B21642EFD099
S214018FB06E4636880700BFB23F1DBE42C5DA80B294
S214018FC0F2BDF0B50200002318001800180023E0D7
S214018FD01E00B6B20C277743EE59360C0700BFB217
S214018FE0D655401C1E00B6B20C277743EE59360AFA
S214018FF00700BFB2D655401C1E00B6B20C277743F9
S214019000ED590600B6B29555401C6406640E05007F
S214019010ADB25455401C5B1C1C00A4B2142C0DDAD6
S2140190202A4D1C00A4B20C266643AC1924790E0006
S214019030B6B20700BFB23F1DBE42C9DA80B2F0BD6C
S21401904010B5002421002249401A04D09D3817D0BB
S2140190502F382CD035E00EE01C48210089B20C22B6
S2140190604A43805880214903884203D2200080B2B7
S214019070FFF71BFF641C200080B21428ECDB20E005
S21401908010E01248210089B20C224A438058114947
S21401909040188021C903884203D2200080B2FFF71E
S2140190A004FF641C200080B21428EADB09E004E017
S2140190B0200080B2FFF7F9FE641C200080B214285D
S2140190C0F6DB10BD00000000A7550020740000204C
S2140190D033FFFF000000C0FF002202604160012153
S2140190E001724272704770B504000E0015002548E3
S2140190F0215A25482018FFF7EFFF7820205C012829
S21401910006D02A00310092B220001830FBF70DFC81
S21401911070BDFEB505000E001400082100226F4642
S2140191203800FEF78BFA2000C0B2782805D0154823
S214019130295A15482818FFF7CFFF7920285C002800
S21401914014D02000C0B211280FD02000C0B21228BF
S2140191500BD02000C0B2312807D02000C0B27E2834
S21401916003D02000C0B27F2800D10AE068467F21E4
S2140191700170467084700322694628001830FBF798
S214019180D4FBF7BD8C100000A810000080207047AB
S21401919010B5010000200200012200E0521C13005D
S2140191A0DBB2052B08DA04239B1ADB000C00DC403B
S2140191B0002CF3D00520801AC0B210BDF8B584B0DB
S2140191C004001300002210001500150016001600FA
S2140191D01600160016006778012F05D122223421C9
S2140191E02000FFF796FF8EE09C46A7687A23E35C93
S2140191F0DB00FB185B786746BFB29BB29F4205D285
S214019200132234212000FFF784FF7CE001910199AD
S21401921089780907090F6B46197001998978C9B2CF
S21401922009096B4659706946097800290BD06946C9
S2140192300978052907D269464978002903D0694685
S2140192404978052905D3312234212000FFF761FF33
S21401925059E0110007E00002019B0F00FFB2DB1985
S214019260DB78C018491C0B006F463F78DBB2BB4267
S214019270F1D30AE02902019B6D462D781700FFB253
S214019280ED195B19DB78CD18521C11006B465B7823
S214019290C9B29942EED3002D05D1222234212000F5
S2140192A0FFF737FF2FE000F087F8280000F087F877
S2140192B0012000F08AF8FFF769FF05002800FFF794
S2140192C067FF02A9742233009BB2CA54761C32008F
S2140192D003011600B6B28B55521C012308E0C61ACC
S2140192E0F7002E00FE401700BFB2CE55521C5B1C85
S2140192F006001F00F6B2FFB2BE42F0D292B202A939
S2140193002000FFF7F0FE05B0F0BD0000002202606D
S2140193104160012101724272704770B504000E006F
S21401932015007948215A79482018FFF7EFFF782071
S214019330205C012806D02A00310092B220001830A5
S214019340FBF7F3FA70BDFEB505000E001400082108
S21401935000226F463800FEF771F92000C0B2782867
S21401936005D06948295A69482818FFF7CFFF7920A0
S214019370285C002814D02000C0B211280FD020008D
S214019380C0B212280BD02000C0B2312807D020006E
S214019390C0B27E2803D02000C0B27F2800D10AE0E8
S2140193A068467F2101704670847003226946280052
S2140193B01830FBF7BAFAF7BD5549086070475549AA
S2140193C0086070475348006870475349087000208A
S2140193D00100524A11700100514A1170514908604A
S2140193E070474D48007870474E4800687047F0B5A2
S2140193F0FFB082B004000E0015000022100069467E
S21401940008808021890001AF3800FEF717F96078DF
S214019410012805D1222236212000FFF794FF6EE0B5
S21401942028000100A2687A23E35CDB00D218527898
S21401943089B292B2914205D2132236212000FFF75B
S21401944082FF5CE034490978012902D002294BD019
S21401945050E0334972780A70304B0A781D78AA4278
S2140194600BD00A781D786D1CEDB2AA4205D0732286
S21401947036212000FFF767FF41E001AA76256F46F7
S2140194803F88D5556D462D886D1C77782E00B6B26F
S21401949097556D1C2A000D781E78B54205D192B2FB
S2140194A001A92000FFF739FF29E01E4D194E376844
S2140194B0BC462F680600B6B2BE19B61E6746B7424E
S2140194C005D2712236212000FFF73DFF17E02E68F6
S2140194D080B2801E301828600878187092B201A9F0
S2140194E02000FFF71AFF0AE0312236212000FFF79D
S2140194F02AFF04E0242236212000FFF724FF7FB054
S21401950002B0F0BD000000008C100000A8100000A2
S2140195105455002058550020AA550020AC5500206F
S214019520AB5500205C5500200022026041600121FD
S21401953001724272704770B504000E00150078483B
S214019540215A78482018FFF7EFFF7820205C012881
S21401955006D02A00310092B220001830FBF7E5F958
S21401956070BDFEB505000E001400082100226F46EE
S2140195703800FEF763F82000C0B2782805D06848A6
S214019580295A68482818FFF7CFFF7920285C002859
S21401959014D02000C0B211280FD02000C0B212286B
S2140195A00BD02000C0B2312807D02000C0B27E28E0
S2140195B003D02000C0B27F2800D10AE068467F2190
S2140195C00170467084700322694628001830FBF744
S2140195D0ACF9F7BDF2B582B00400150008210026EB
S2140195E032006F463800FEF729F83000A0687A216D
S2140195F0615CC90040184078ADB280B2854205D2A0
S214019600132228212000FFF7ACFF86E060780128AE
S21401961005D1222228212000FFF7A3FF7DE0029832
S21401962041784906490E80786A466823137051705E
S214019630C9B2002905D0022936D01BD303294DD043
S21401964066E00100C9B2012906D00100C9B20229AB
S21401965002D0C0B2032807D13348067002226946F9
S2140196602000FFF768FF04E0312228212000FFF7E1
S21401967078FF52E00100C9B2012906D00100C9B243
S214019680022902D0C0B2032808D101202649087059
S214019690022269462000FFF74EFF04E0312228210E
S2140196A02000FFF75EFF38E00100C9B2012906D0AD
S2140196B00100C9B2022902D0C0B2032808D1022093
S2140196C019490870022269462000FFF734FF04E0BA
S2140196D0312228212000FFF744FF1EE00100C9B215
S2140196E0012906D00100C9B2022902D0C0B203285E
S2140196F008D103200C490870022269462000FFF7B2
S2140197001AFF04E0312228212000FFF72AFF04E097
S214019710122228212000FFF724FFF7BD00000000D9
S2140197208C100000A8100000A955002001010100BE
S2140197302B010100D901010000000000F901010020
S214019740CD0201004D040100A10401005B050100EA
S214019750AF05010075060100C90601008907010071
S214019760DD07010097080100EB080100A5090100CB
S214019770F9090100B90A0100090B0100670B010094
S2140197809F0B0100CB0B0100050C0100350C0100FD
S214019790CF0C0100750D0100CB0E0100AD110100CB
S2140197A000000000B5110100D7110100FD110100F4
S2140197B01F12010045120100000000004F120100B7
S2140197C097120100291301004F13010075130100C0
S2140197D09B130100C1130100E71301000D140100E2
S2140197E033140100591401007F140100A51401006F
S2140197F073150100BF1601001B170100E1170100D8
S2140198003D180100F1180100271901007519010022
S214019810AB190100F3190100291A0100751A01009C
S214019820AB1A0100F31A0100291B0100751B010088
S214019830AD1B0100F51B0100131C0100391C0100C2
S214019840571C01007D1C01009B1C0100C11C01006E
S214019850DF1C0100051D0100231D0100491D01003B
S214019860671D01008D1D0100171E0100F71E010076
S214019870151F01003B1F01008B1F01001120010075
S21401988061200100F120010041210100C7210100F2
S214019890172201009D220100ED2201007323010021
S2140198A0C32301004D240100DB240100A52501008E
S2140198B0A9250100CF250100ED2501001326010091
S2140198C0312601005726010077260100A126010056
S2140198D0C1260100EB2601000B27010035270100F8
S2140198E0552701007F27010000000000872701009F
S2140198F0000000008F2701000000000097270100EC
S214019900F5270100D12801002F2901000B2A0100AB
S214019910392A01008B2A0100B92A0100112B010006
S214019920312B010000220260416001210172427266
S214019930704770B504000E0015002548215A2548C9
S2140199402018FFF7EFFF7820205C012806D02A00B8
S214019950310092B220001830FAF7E7FF70BDFEB56D
S21401996005000E001400082100226F463800FDF79E
S21401997065FE2000C0B2782805D01548295A15483A
S2140199802818FFF7CFFF7920285C002814D0200084
S214019990C0B211280FD02000C0B212280BD0200070
S2140199A0C0B2312807D02000C0B27E2803D02000E4
S2140199B0C0B27F2800D10AE068467F210170467058
S2140199C084700322694628001830FAF7AEFFF7BD07
S2140199D08C100000A8100000F2B582B0040015003B
S2140199E0002630003000082132006F463800FDF7AF
S2140199F025FE2800A1687A22A25CD200891849783F
S214019A0080B289B2884205D213222E212000FFF7A8
S214019A10A6FF7BE0029841780902827811436A46E4
S214019A206E231370437853708378937000E0761C2E
S214019A303200A38A92B29A4263D2226933009BB261
S214019A4014275F43D25B0B009BB29A42EFD1216988
S214019A50320092B214235343C918097900290FD052
S214019A60A178226933009BB214275F43D219127979
S214019A70914205D0332222212000FFF770FF45E0F6
S214019A80ADB2E91E226933009BB214255D4352191B
S214019A909289914205D013222E212000FFF75FFF05
S214019AA034E02169320092B214235343C9188978ED
S214019AB0032909D06178226933009BB214255D43DE
S214019AC05219D278914205D222222E212000FFF788
S214019AD046FF1BE02169320092B214235343C91892
S214019AE08A89C11C2069B6B214237343C0188568DD
S214019AF02800FDF795FD032269462000FFF719FFB0
S214019B0004E031222E212000FFF729FFF7BD0000D7
S214019B10002202604160012101724272704770B5F5
S214019B2004000E0015002548215A25482018FFF785
S214019B30EFFF7820205C012806D02A00310092B27F
S214019B4020001830FAF7F1FE70BDFEB505000E00D4
S214019B501400082100226F463800FDF76FFD200033
S214019B60C0B2782805D01548295A15482818FFF795
S214019B70CFFF7920285C002814D02000C0B211281D
S214019B800FD02000C0B212280BD02000C0B231285E
S214019B9007D02000C0B27E2803D02000C0B27F28A4
S214019BA000D10AE068467F21017046708470032266
S214019BB0694628001830FAF7B8FEF7BD8C10000089
S214019BC0A8100000F8B5FFB081B005000C00170022
S214019BD000221000100010001000802189006E463F
S214019BE03000FDF72BFD3800A9687A22AA5CD20066
S214019BF08918497880B289B2884205D21322192180
S214019C002800FFF7A2FF5EE020007F264178314062
S214019C106C46592222706170C9B2012904D002290A
S214019C201DD00A2934D049E0BFB2032F05D0132234
S214019C3019212800FFF789FF45E08078C0B2FFF7B9
S214019C4062F9A6700121E170010089B2090A217149
S214019C506071062269462800FFF761FF33E0BFB254
S214019C60032F05D0132219212800FFF76EFF2AE0E3
S214019C708278A670D2B2FF21FE31E01CFFF75EF9B2
S214019C80C01C020092B269462800FFF748FF1AE09E
S214019C90BFB2022F05D0132219212800FFF755FF66
S214019CA011E0FF21FE31E01CFFF78BF9C01C02001A
S214019CB092B269462800FFF732FF04E0122219210A
S214019CC02800FFF742FF7FB002B0F0BD002202601D
S214019CD04160012101724272704770B504000E00A6
S214019CE015005748215A57482018FFF7EFFF7820EC
S214019CF0205C012806D02A00310092B220001830DC
S214019D00FAF713FE70BDFEB505000E00140008211B
S214019D1000226F463800FDF791FC2000C0B278287B
S214019D2005D04748295A47482818FFF7CFFF79201A
S214019D30285C002814D02000C0B211280FD02000C3
S214019D40C0B212280BD02000C0B2312807D02000A4
S214019D50C0B27E2803D02000C0B27F2800D10AE01E
S214019D6068467F2101704670847003226946280088
S214019D701830FAF7DAFDF7BDF2B582B00400150027
S214019D800821002632006F463800FDF757FCA06810
S214019D907A21615CC90040184078ADB280B2854234
S214019DA005D0132210212000FFF7ADFF47E00298EF
S214019DB040784006400E694650220A704870224A92
S214019DC0A25A92B2120A8A701F4AA25ACA701F4A2F
S214019DD0A25A92B2120A0A711C4AA25A4A71010088
S214019DE0C9B2012906D025D303290BD012D30429E1
S214019DF018D01FE0A6706070062269462000FFF7A3
S214019E006CFF1CE0A6706070062269462000FFF712
S214019E1064FF14E0A6706070062269462000FFF712
S214019E205CFF0CE0A6706070062269462000FFF712
S214019E3054FF04E0122210212000FFF764FFF7BD53
S214019E408C100000A8100000881000008A10000086
S214019E50002202604160012101724272704770B5B2
S214019E6004000E0015002548215A25482018FFF742
S214019E70EFFF7820205C012806D02A00310092B23C
S214019E8020001830FAF751FD70BDFEB505000E0032
S214019E901400082100226F463800FDF7CFFB200092
S214019EA0C0B2782805D01548295A15482818FFF752
S214019EB0CFFF7920285C002814D02000C0B21128DA
S214019EC00FD02000C0B212280BD02000C0B231281B
S214019ED007D02000C0B27E2803D02000C0B27F2861
S214019EE000D10AE068467F21017046708470032223
S214019EF0694628001830FAF718FDF7BD8C100000E7
S214019F00A8100000FEB50400160000221500082166
S214019F106F463800FDF792FB6078012805D12222B2
S214019F2037212000FFF7B1FF3EE0A0687A21615C8F
S214019F30C90040184078B6B280B2864205D21322D4
S214019F4037212000FFF7A1FF2EE0772069462A007F
S214019F5092B288546D1CFFF744FA012802D00228F9
S214019F6014D019E0FFF740FA0600FFF72BFA8642F5
S214019F7005D0132237212000FFF787FF11E02A00C2
S214019F8092B269462000FFF76AFF0AE031223721C4
S214019F902000FFF77AFF04E0242237212000FFF794
S214019FA074FF0020FFF711FAF7BD000000220260DF
S214019FB04160012101724272704770B504000E00C3
S214019FC015002548215A25482018FFF7EFFF78206D
S214019FD0205C012806D02A00310092B220001830F9
S214019FE0FAF7A3FC70BDFEB505000E0014000821AB
S214019FF000226F463800FDF721FB2000C0B278280A
S21401A00005D01548295A15482818FFF7CFFF79209B
S21401A010285C002814D02000C0B211280FD02000E0
S21401A020C0B212280BD02000C0B2312807D02000C1
S21401A030C0B27E2803D02000C0B27F2800D10AE03B
S21401A04068467F21017046708470032269462800A5
S21401A0501830FAF76AFCF7BD8C100000A810000053
S21401A060FEB504000D001600082100226F463800D8
S21401A070FDF7E4FAA0687A21615CC90040184078CF
S21401A080B6B280B2864205D2132285212000FFF7A0
S21401A090AAFF2CE06078012805D122228521200024
S21401A0A0FFF7A1FF23E068784006400E6946C52207
S21401A0B00A704870C0B2012802D0022809D011E007
S21401A0C00120FEF7EFFE022269462000FFF775FF2A
S21401A0D00DE00020FEF7E6FE022269462000FFF7AB
S21401A0E06CFF04E0122285212000FFF77CFFF7BDFC
S21401A0F0002202604160012101724272704770B510
S21401A10004000E0015002548215A25482018FFF79F
S21401A110EFFF7820205C012806D02A00310092B299
S21401A12020001830FAF701FC70BDFEB505000E00E0
S21401A1301400082100226F463800FDF77FFA200040
S21401A140C0B2782805D01548295A15482818FFF7AF
S21401A150CFFF7920285C002814D02000C0B2112837
S21401A1600FD02000C0B212280BD02000C0B2312878
S21401A17007D02000C0B27E2803D02000C0B27F28BE
S21401A18000D10AE068467F21017046708470032280
S21401A190694628001830FAF7C8FBF7BD8C10000096
S21401A1A0A8100000FEB504000D00160008210022CC
S21401A1B06F463800FDF742FAFF20A1687A22A25CBA
S21401A1C0D20089184978B6B289B28E4205D01322D8
S21401A1D011212000FFF7A9FF2AE069784906490EF8
S21401A1E06A465123137051709070C9B2012904D088
S21401A1F019D303290FD008D315E00322694620009E
S21401A200FFF77DFF00F04DF812E0032269462000BB
S21401A210FFF775FF0CE0032269462000FFF76FFF8A
S21401A22000F045F804E0122211212000FFF77DFF1F
S21401A230F7BD000010B50400102220492000FDF7EC
S21401A240EFF910BD10B50400C02104222000FDF76F
S21401A250E7F910BD70B504000C22194D2900103124
S21401A26026003000FDF7DCF90822291D25000C35F3
S21401A2702800FDF7D5F92020E07270BD10B5040066
S21401A280C0200822011D2000FDF7CAF910BD10B537
S21401A2900400C0200822010028312000FDF7C0F983
S21401A2A010BD80B523210748FAF7E4FD01BD80B54E
S21401A2B023210448FAF7DEFD01BD0000E00001009D
S21401A2C0C0000100D031002000B5017A00290FD06E
S21401A2D0417A00290CD101684268914208D201688E
S21401A2E0491C016001684268914201D10121417215
S21401A2F000BD10B5040084204001201803C80022C8
S21401A300401C514184225201A21803C2083A2F4828
S21401A3102018FFF7D9FF2E482018FFF7D5FF2D4844
S21401A3202018FFF7D1FF10BD2B482C490860704755
S21401A3302B4803C8704780B52A480168491C01604C
S21401A340274A03CA083A0023401C594103C2083A67
S21401A3502548FFF7CEFF01BD80B52449224800F00D
S21401A36051F8FDF793F901BD10B51E4C2068002881
S21401A3702BD01D484078022805D1FFF7D5FF2321B1
S21401A3801B48FAF777FD2068401E2060194C2068AC
S21401A390401C206018480168491C0160FDF7BBF9A4
S21401A3A0FCF7F0F920680521F8F76BFC002904D1C9
S21401A3B0FBF722FD1148FCF736F820682068206874
S21401A3C00F49884201D30020206010BD9010000084
S21401A3D09C100000A810000055AAAA55F0630020A2
S21401A3E000200020443200200820002040000020E9
S21401A3F0D0310020483200204C320020403200206C
S21401A4001027000010B504002000FDF745FA0548A6
S21401A410A0600548E0600F206060044820610620C7
S21401A420A08210BDF0A80100A0AB0100C801002069
S21401A43080B50800FFF722FF01BD4078087070471D
S21401A44080B50800FFF723FF01BD80B50800FFF7C0
S21401A450F9FE01BD80B50800FFF7ECFE01BD80B531
S21401A4600800FFF7F7FE01BD0022026041600121EE
S21401A47001724272704770B504000E001500444820
S21401A480215A44482018FFF7EFFF7820205C012866
S21401A49006D02A00310092B220001830FAF745FAA9
S21401A4A070BDFEB505000E001400082100226F469F
S21401A4B03800FDF7C3F82000C0B2782805D034482C
S21401A4C0295A34482818FFF7CFFF7920285C00283E
S21401A4D014D02000C0B211280FD02000C0B212281C
S21401A4E00BD02000C0B2312807D02000C0B27E2891
S21401A4F003D02000C0B27F2800D10AE068467F2141
S21401A5000170467084700322694628001830FAF7F5
S21401A5100CFAF7BDFEB504000D00160000220292EB
S21401A52008216F463800FDF789F8A0687A21615C3A
S21401A530C90040184078B6B280B2864205D01322D0
S21401A54014212000FFF7ADFF20E00299687800048F
S21401A5500843A97809020143E878084354216A466A
S21401A560117001000C4A891A03D09D3901D02F3988
S21401A57007D1FEF765FD012269462000FFF77BFF44
S21401A58004E0312214212000FFF78BFFF7BD000005
S21401A5908C100000A810000033FFFF0000220260AC
S21401A5A04160012101724272704770B504000E00CD
S21401A5B015002548215A25482018FFF7EFFF782077
S21401A5C0205C012806D02A00310092B22000183003
S21401A5D0FAF7ABF970BDFEB505000E0014000821B0
S21401A5E000226F463800FDF729F82000C0B278280F
S21401A5F005D01548295A15482818FFF7CFFF7920A6
S21401A600285C002814D02000C0B211280FD02000EA
S21401A610C0B212280BD02000C0B2312807D02000CB
S21401A620C0B27E2803D02000C0B27F2800D10AE045
S21401A63068467F21017046708470032269462800AF
S21401A6401830FAF772F9F7BD8C100000A810000058
S21401A650FEB504000D001600082100226F463800E2
S21401A660FCF7ECFFA0687A21615CC90040184078CD
S21401A670B6B280B2864205D013223E212000FFF7F3
S21401A680AAFF15E068784006400E0100C9B200290D
S21401A69009D169467E220A70487002226946200066
S21401A6A0FFF783FF04E012223E212000FFF793FF0D
S21401A6B0F7BD0000E7690100D1690100BB6901002F
S21401A6C0A5690100536A01003D6A0100276A01007D
S21401A6D0116A0100000000000000000000000000F8
S21401A6E000000000BF6A0100A96A0100936A010028
S21401A6F07D6A01000000000000000000000000006C
S21401A70000000000E96A01000000000000000000EF
S21401A71000000000556B01003F6B0100296B010032
S21401A720136B0100C16B0100AB6B0100956B01005F
S21401A7307F6B010000000000000000000000000028
S21401A7400000000000000000000000000000000003
S21401A75000000000EB6B010000000000000000009C
S21401A76000000000000000000000000000000000E3
S21401A77000000000676C0100516C0100316C0100A3
S21401A780156C0100916C0100000000000000000043
S21401A79000000000FFB51F481F49204A0392204AC7
S21401A7A0204B214C0294214C214D0195214D224EE6
S21401A7B0224F009703E00F780770401C491C039F47
S21401A7C08F42F8D10298984207D018781070521C20
S21401A7D05B1CF7E700202070641C0198A042F9D1A9
S21401A7E00098B04204D030782870761C6D1CF7E7CC
S21401A7F0002006E0124982008958124A8300D1508F
S21401A800401C114989088842F4D30E480F49086054
S21401A810FFBD00BF00000020648C0100A48E010073
S21401A82040020020C4AC0100C4AC0100002000209E
S21401A830AD550020000000000000000000000000F0
S21401A84000000100000001000000000008ED00E02B
S21401A85000000100310700000001080001000000AF
S21401A860FFFFFFFF01000100DF07000000010800F5
S21401A87001000000FFFFFFFF02000100440400008A
S21401A8800001080001000000FFFFFFFF03000100B8
S21401A890550500000001080001000000FFFFFFFF52
S21401A8A005000100B10700000000080000000000DC
S21401A8B0FFFFFFFF06000100010200000000080084
S21401A8C000000000FFFFFFFF07000100220200005A
S21401A8D00000080000000000FFFFFFFF000000006E
S21401A8E00000000000000000000000000000000062
S21401A8F010020100799D010011020100A5A10100CD
S21401A900270201005981010028030100D5950100A5
S21401A9103E02010051A601008502010061A001006E
S21401A92022030000BD8701002E040000D999010012
S21401A9301404000015A5010019030100C59B0100C0
S21401A9402F030000A18A010031040100E584010003
S21401A95034050000BD91010036020000EF930100AE
S21401A96037010000059F010072B600210022002376
S21401A9700024002500260027B846B946BA46BB463D
S21401A980BC460C490C4A521A013A05DD0020042344
S21401A99008601944043AFBDA0848854608488047A7
S21401A9A00848804762B600F00FF8804700F01AF8B2
S21401A9B0FEE7000000000020FF630020F05F00209B
S21401A9C0B368010095A701000548014603B468462F
S21401A9D080F3098800BF00BF00BF00BF00F016F873
S21401A9E0A5EDF5FE80B5FBF755FFFBF778F8FDF70B
S21401A9F0FBFA05490020FDF7FDF9FBF73DFFFFF7E0
S21401AA00ABFCFFF7B1FCFCE790AC010000F00DF8E1
S21401AA10002801D000BF00BF00BF00BF002000BF5C
S21401AA2000BFFFF7DFFF00F002F80120704780B596
S21401AA3000F002F801BD00000746384600F002F8B3
S21401AA40FBE7000080B500BF00BF024A11001820D6
S21401AA50ABBEFBE72600020046697273742066727D
S21401AA60616D652073686F756C64206E6F742075F8
S21401AA707365206D756C7469706C65206672616DA6
S21401AA8065207472616E736D697373696F6E2E00E3
S21401AA904D756C74692D6672616D65207265737093
S21401AAA06F6E736520746F6F206C617267652066C8
S21401AAB06F7220726563656976696E672062756676
S21401AAC06665722E000000008D690100F9690100BB
S21401AAD000000000656A010000000000D16A010064
S21401AAE0FB6A0100676B0100000000000000000027
S21401AAF0D36B010000000000FD6B0100796C0100C2
S21401AB0095690100016A0100000000006D6A0100FC
S21401AB1000000000D96A0100036B01006F6B0100A1
S21401AB200000000000000000DB6B010000000000D8
S21401AB30056C0100816C01004D65737361676520CA
S21401AB4073697A6520746F6F206C617267652E2059
S21401AB505365742061206C61726765722073656E3F
S21401AB6064206275666665720A00000041626F7253
S21401AB70742070726576696F7573206D6573736185
S21401AB8067652C207472616E736D697373696F6E7D
S21401AB9020696E2070726F67726573732E0A0000EB
S21401ABA0000000000000000000000000000000009F
S21401ABB0000000000000000000000000000000008F
S21401ABC0000000000000000000000000000000007F
S21401ABD053696E676C652D6672616D65206C656E76
S21401ABE067746820746F6F20736D616C6C206F7270
S21401ABF020746F6F206C617267652E0046697273F0
S21401AC0074206672616D652073686F756C6420626E
S21401AC1065203820627974657320696E206C656ED4
S21401AC206774682E00000000436F6E736563757469
S21401AC30697665206672616D6520746F6F20736832
S21401AC406F72742E00000000466C6F7720636F6E83
S21401AC5074726F6C206672616D6520746F6F2073FD
S21401AC60686F72742E000000B7740100A1740100B1
S21401AC708B74010075740100DF740100C974010052
S21401AC80303132333435363738394142434445461C
S21401AC906170702073746172740A00005465726D7D
S21401ACA0696E616C000000000001020304050000EB
S21401ACB0534547474552000030280000010203046F
S20801ACC0000000008A
S80401A9C988
